:100000000C9463000C948B000C948B000C948B006C
:100010000C948B000C947D1F0C948B000C948B0023
:100020000C948B000C948B000C948B000C948B0024
:100030000C948B000C948B000C948B000C948B0014
:100040000C94141E0C948B000C94E21D0C94BC1D9B
:100050000C948B000C948B000C948B000C948B00F4
:100060000C945E1E0C948B000000000024002700FE
:100070002A0000000000250028002B0000000000DE
:1000800023002600290004040404040404040202DA
:100090000202020203030303030301020408102007
:1000A0004080010204081020010204081020000012
:1000B0000008000201000003040700000000000027
:1000C0000000F81F033011241FBECFEFD8E0DEBFC1
:1000D000CDBF27E0A6EBB4E001C01D92A631B20768
:1000E000E1F714E0A0E0B1E0ECE5FEE602C0059027
:1000F0000D92A63BB107D9F710E0C2E6D0E004C0EC
:100100002197FE010E942035C136D107C9F70E9410
:10011000D6200C9421370C940000982F2091D905FB
:1001200081E0213208F043C08091B5058111FCCFF8
:100130008091D80532E03093B5059093B4059FEFD8
:100140009093B3051092B2052093B105A8EBB5E0EA
:10015000E1E9F5E090E0291331C01092900590910B
:100160009005880F892B8093900580918F058130B1
:1001700049F510928F05809190058093BB00809186
:10018000BC0083FDF8CF85EC8093BC008091B50561
:100190008230E1F38091B3058F3FB1F08091B305D8
:1001A0008032A1F08091B305803391F084E0109209
:1001B000B7051092D9051092B60508953D91319377
:1001C0009F5FC9CF85EEE0CF80E0F1CF82E0EFCF37
:1001D00083E0EDCF80916D0590916E05891B990BA1
:1001E0000895089508952F923F924F925F926F92D3
:1001F0007F928F929F92AF92BF92CF92DF92EF92B7
:10020000FF920F931F93CF93DF93CDB7DEB76C9719
:100210000FB6F894DEBF0FBECDBF522E3D874E877E
:10022000252E462E372E782E692EA982BF86C88AA3
:10023000D98AEA8AFB8A0C8B1D8B988E8F8A2115AE
:1002400000EA30070CEA400709EB500703E06007BB
:1002500071058105910509F098F52F3F10EE3107E2
:1002600015EF410715E051076105710581059105FD
:1002700009F008F40BC12F3F354D41415E47634003
:1002800071058105910509F008F40BC129813F85AD
:10029000488959896A897B898C899D89A0E099243C
:1002A00093940E940035C9F4F1E0FE8B04E0802EA7
:1002B000912CA12CB12C89869A86AB86BC8616C15E
:1002C000512CB0EABD87ECEAEE8789EB282E93E04B
:1002D000492E312C712C612CD9CFA52CBD84CE8414
:1002E000D22CE42CF32C072D162D29813F8548892B
:1002F00059896A897B898C899D890E944B34298719
:100300003A874B875C8729853A854B855C85B6E0C3
:10031000AB2EB12C263031054105510568F0898599
:100320009A85AB85BC8589309740A105B105E0F081
:10033000F8E0AF2EA7E0BA2EC12CD12CE12CF12C85
:1003400000E010E029813F85488959896A897B89C5
:100350008C899D890E944B34522E3D874E87252ED5
:10036000462E372E782E692EA52CBD84CE84D22C15
:10037000E42CF32C072D162D29813F8548895989B6
:100380006A897B898C899D890E944934AA24AA9410
:10039000BB24BA94EFE0CE2ED12CE12CF12C00E05E
:1003A00010E00E948633A52CBD84CE84D22CE42C90
:1003B000F32C072D162D0E944B34A32FF42FE52F7D
:1003C000422F5A2F6F2F7E2FCC24CA94DC2C8FE023
:1003D000E82EF12C411551056105710521F4C12C60
:1003E000D12C7601C394AA24A3949A1409F4E5C0ED
:1003F00001E00E8BCB01BA0137E0660F771F881F33
:10040000991F3A95D1F7A70196010E944533298F8C
:100410003A8F4B8F5C8F89849A84AB84BC8447E08D
:10042000880C991CAA1CBB1C4A95D1F79501840124
:1004300012502109310948015901298D3A8D4B8DFE
:100440005C8D280D391D4A1D5B1DAF89B88D2D931C
:100450003D934D935C931397FD016483758386836D
:1004600097831896CD92DD92ED92FC921B978E8821
:10047000882009F481C059829D849F86AE84A88A11
:10048000298A4A8A3B8A7C8A6D8A76C0512C01EE81
:100490000D8715EF1E8725E0222E412C312C712C63
:1004A000612C29813F85488959896A897B898C8992
:1004B0009D89A0E0912C0E94003509F00ECFA52C5B
:1004C000BD84CE84D22CE42CF32C072D162D20E0F5
:1004D00034E04BE654EF64E170E080E090E00E948D
:1004E0004B3429873A874B875C871E8A89849A8494
:1004F000AB84BC84A501940160E070E0CB01A52C25
:10050000BD84CE84D22CE42CF32C072D162D298308
:100510003A834B835C836D837E838F83988760E00F
:1005200070E080E090E00E94863329833F87488B0B
:10053000598B6A8B7B8B8C8B9D8B0E89C12CD12C1C
:100540007601C39440E050E0BA01013009F052CF87
:10055000AF89B88D1D921D921D921C921397FD01BB
:10056000148215821682178281E090E0A0E0B0E04C
:1005700080879187A287B38729813F8548895989D8
:100580006A897B898C899D896C960FB6F894DEBF49
:100590000FBECDBFDF91CF911F910F91FF90EF90D4
:1005A000DF90CF90BF90AF909F908F907F906F9093
:1005B0005F904F903F902F900895AF89B88D1D9216
:1005C0001D921D921C921397FD01148215821682B2
:1005D000178281E090E0A0E0B0E080879187A28759
:1005E000B3875982FD85FF878E84888A49CFDF9241
:1005F000EF92FF920F931F93CF93DF93FC01E08064
:10060000F18002811381D481C581B681D7809701A1
:10061000A8016D2F7C2F8B2F9D2D35534C405109F8
:1006200061097109810991092F3F34434C405105FB
:10063000610571058105910509F0D0F49701A801C4
:100640006D2F7C2F8B2F9D2D07E00E94B8342083C7
:10065000318342835383648375838683978387E0E2
:10066000DF91CF911F910F91FF90EF90DF90089550
:100670009701A8016D2F7C2F8B2F9D2D3A56484155
:10068000510961097109810991092F3F3946484192
:100690005105610571058105910509F098F49701EF
:1006A000A8016D2F7C2F8B2F9D2D06E00E94B83462
:1006B0002083318342835383648375838683978346
:1006C00086E0CECF9701A8016D2F7C2F8B2F9D2D1B
:1006D000345D4043510961097109810991092F3F36
:1006E000334D40435105610571058105910509F0C0
:1006F00098F49701A8016D2F7C2F8B2F9D2D05E07D
:100700000E94B8342083318342835383648375838A
:100710008683978385E0A4CF9701A8016D2F7C2F56
:100720008B2F9D2D385A4146510961097109810964
:1007300091092F3F374A41465105610571058105F1
:10074000910509F098F49701A8016D2F7C2F8B2F4C
:100750009D2D04E00E94B83420833183428353836B
:10076000648375838683978384E07ACF9701A80199
:100770006D2F7C2F8B2F9D2D3055434C51096109D6
:100780007109810991092F3F3F44434C510561058F
:1007900071058105910509F098F49701A8016D2F65
:1007A0007C2F8B2F9D2D03E00E94B8342083318352
:1007B00042835383648375838683978383E050CF1A
:1007C0009701A8016D2F7C2F8B2F9D2D305A464805
:1007D000514061097109810991092F3F3F494648FC
:1007E0005140610571058105910509F098F4970163
:1007F000A8016D2F7C2F8B2F9D2D02E00E94B83415
:1008000020833183428353836483758386839783F4
:1008100082E026CF9701A8016D2F7C2F8B2F9D2D75
:1008200030544D40534061097109810991092F3FAE
:100830003F434D405340610571058105910509F025
:1008400098F49701A8016D2F7C2F8B2F9D2D01E02F
:100850000E94B83420833183428353836483758339
:100860008683978381E0FCCE80E0FACE0895AF9234
:10087000BF92CF92DF92EF92FF920F931F93CF938D
:10088000DF936C017B018B01040F151FEB015E01EF
:10089000AE18BF08C017D10759F06991D601ED9184
:1008A000FC910190F081E02DC6010995892B79F723
:1008B000C501DF91CF911F910F91FF90EF90DF90D5
:1008C000CF90BF90AF900895FC0144815581608125
:1008D00071818AEF96E00C943704FC01538D448DAE
:1008E000252F30E0842F90E0821B930B541710F0DB
:1008F000CF96089501970895FC01918D828D9817E8
:1009000061F0A28DAE0FBF2FB11D5D968C91928DBF
:100910009F5F9F73928F90E008958FEF9FEF0895F0
:10092000FC01918D828D981731F0828DE80FF11DB9
:10093000858D90E008958FEF9FEF0895FC01918DD4
:10094000228D892F90E0805C9F4F821B91098F73CD
:10095000992708958AED95E00E949E0421E0892B55
:1009600009F420E0822F089580E090E0892B29F09F
:100970000E94AA0481110C9400000895FC01A48D2A
:10098000A80FB92FB11DA35ABF4F2C91848D90E0B1
:1009900001968F739927848FA689B7892C93A08994
:1009A000B1898C91837080648C93938D848D98131E
:1009B00006C00288F389E02D80818F7D80830895B1
:1009C000EF92FF920F931F93CF93DF93EC0181E09F
:1009D000888F9B8D8C8D98131AC0E889F989808146
:1009E00085FF15C09FB7F894EE89FF896083E88979
:1009F000F98980818370806480839FBF81E090E06B
:100A0000DF91CF911F910F91FF90EF900895F62EF7
:100A10000B8D10E00F5F1F4F0F731127E02E8C8D91
:100A20008E110CC00FB607FCFACFE889F9898081D6
:100A300085FFF5CFCE010E94BE04F1CFEB8DEC0F08
:100A4000FD2FF11DE35AFF4FF0829FB7F8940B8FF3
:100A5000EA89FB8980818062CFCFCF93DF93EC015D
:100A6000888D8823B9F0AA89BB89E889F9898C9196
:100A700085FD03C0808186FD0DC00FB607FCF7CF52
:100A80008C9185FFF2CF808185FFEDCFCE010E9452
:100A9000BE04E9CFDF91CF910895833081F028F42F
:100AA000813099F08230A9F008958730A9F088301C
:100AB000C9F08430B1F4809180008F7D03C08091B3
:100AC00080008F7780938000089584B58F7784BDF0
:100AD000089584B58F7DFBCF8091B0008F77809390
:100AE000B00008958091B0008F7DF9CFCF93DF9350
:100AF000282F30E0F901E255FF4F8491F901E656C5
:100B0000FF4FD491F901EA57FF4FC491CC23A1F0D4
:100B100081110E944D05EC2FF0E0EE0FFF1FE4580D
:100B2000FF4FA591B491EC91ED2381E090E009F4A1
:100B300080E0DF91CF91089580E090E0FACF1F939D
:100B4000CF93DF93282F30E0F901E255FF4F8491D6
:100B5000F901E656FF4FD491F901EA57FF4FC491CE
:100B6000CC23A9F0162F81110E944D05EC2FF0E047
:100B7000EE0FFF1FEE58FF4FA591B4918FB7F89479
:100B8000EC91111108C0D095DE23DC938FBFDF916B
:100B9000CF911F910895DE2BF8CF10926E05109221
:100BA0006D051092B7051092D9051092B50581E038
:100BB0008093B40510928F0561E082E10E949F0549
:100BC00061E083E10E949F05E9EBF0E080818E7F88
:100BD000808380818D7F808388E48093B80085E462
:100BE0008093BC0081EF90E090936C0580936B053F
:100BF00082EF90E090936A05809369050895CF9302
:100C0000DF9390E0FC01E656FF4F24918A579F4FF7
:100C1000FC0184918823C9F090E0880F991FFC01A2
:100C2000E859FF4FA591B491FC01EE58FF4FC591D3
:100C3000D49161110DC09FB7F8948C9120958223B7
:100C40008C938881282328839FBFDF91CF910895BB
:100C5000623051F49FB7F8943C91822F80958323A2
:100C60008C93E8812E2BEFCF8FB7F894EC912E2B3D
:100C70002C938FBFEACF8E50806480937C0080914C
:100C80007A00806480937A0080917A0086FDFCCFA0
:100C9000809178009091790008953FB7F894809101
:100CA000020590910305A0910405B091050526B5B4
:100CB000A89B05C02F3F19F00196A11DB11D3FBF94
:100CC000BA2FA92F982F8827BC01CD01620F711D63
:100CD000811D911D42E0660F771F881F991F4A955D
:100CE000D1F708958F929F92AF92BF92CF92DF92E9
:100CF000EF92FF924B015C010E944D066B017C015B
:100D00000E944D066C197D098E099F09683E73404B
:100D100081059105A8F321E0821A9108A108B10884
:100D200088EEC80E83E0D81EE11CF11C81149104EA
:100D3000A104B10429F7FF90EF90DF90CF90BF900E
:100D4000AF909F908F9008952FB7F8946091FE0414
:100D50007091FF0480910005909101052FBF0895C7
:100D600085ED8093BC008091BC0084FDFCCF109287
:100D7000B50508952091DA04260F3327331F213259
:100D80003105ECF42091B505FC0190E080E02430C1
:100D900069F082E00895A091DA042191AC014654F3
:100DA0005B4FA40FB52FB11D2C930196861798F3B6
:100DB0008091DA04680F6093DA0480E0089581E09E
:100DC00008950895E0916E0580916D05E81730F45F
:100DD000F0E0E159FA4F808190E008958FEF9FEFA6
:100DE000089590916E0580916D052FEF3FEF981754
:100DF00048F4E92FF0E0E159FA4F208130E09F5F9D
:100E000090936E05C9010895CF92DF92EF92FF9201
:100E10000F931F93CF93DF937C01CB018A01209125
:100E2000B605222389F0EB016B01C40ED51ECC154B
:100E3000DD0569F06991D701ED91FC910190F08198
:100E4000E02DC7010995F3CF642F0E94BA06C801AF
:100E5000DF91CF911F910F91FF90EF90DF90CF9096
:100E60000895CF93DF931F92CDB7DEB769832091AA
:100E7000B6052223F9F02091D905203258F021E05F
:100E800030E0FC013383228390E080E00F90DF911B
:100E9000CF9108958091B705E82FF0E0E854FA4F1C
:100EA000998190838F5F8093B7058093D90581E006
:100EB00090E0ECCF61E0CE0101960E94BA06F7CF38
:100EC000CF93C62F91E09093B60590E69093D80506
:100ED0001092B7051092D905682F87E796E00E9417
:100EE00031076C2F87E796E00E94310781E0CF91B0
:100EF0000C948D000F931F93CF93DF938B0191E0A0
:100F00009093B60590E69093D8051092B70510928D
:100F1000D905682F87E796E00E943107E801085F4E
:100F20001F4F699187E796E00E943107C017D107EC
:100F3000C1F781E0DF91CF911F910F910C948D004B
:100F400090E080E008958FE00E943B0690933F057B
:100F500080933E05BC01990F880B990B0E94853048
:100F600020E030E040EA50E40E94E43020E030E04D
:100F700040E85AE30E94E4306093B6047093B704EB
:100F80008093B8049093B9040895CF93DF9391E0D0
:100F90009093B60590E69093D8051092B7051092FD
:100FA000D905682F87E796E00E94310781E00E940B
:100FB0008D008091B5058111FCCF81E08093B5054E
:100FC0001092B4059FEF9093B3051092B205109262
:100FD000B1058093900580919005806C8093900579
:100FE00080918F05813061F510928F058091900579
:100FF0008093BB008091BC0083FDF8CF85EC80938B
:10100000BC008091B5058130E1F38091B20581117A
:1010100019C08091B205E1E9F5E0AFE6B5E0C0E0C6
:10102000C81312C010926E05C0936D0580916E05B5
:10103000C81771F087E796E00E94F106D82FF6CF27
:1010400085EEDDCF81E0E7CF91919D93CF5FE8CF33
:101050008D2FDF91CF910895CF93C0E1C80F8C2FD2
:101060000E94C507682F63608C2FCF910C94600796
:10107000CF93DF93D82FC62F83E00E94C50761E08E
:1010800070E001C0660FDA95EAF7C13039F4609577
:10109000682383E0DF91CF910C946007682BF9CF30
:1010A0000F931F93CF938B01C0E1C80F8C2F0E9429
:1010B000C507682F012B39F46F7D8C2FCF911F91BD
:1010C0000F910C9460076062F8CFCF93DF93EC012F
:1010D00060E08E810E949F0561E08E810E949F05E5
:1010E00060E08E810E949F058BE891E00197F1F707
:1010F000DF91CF910895CF92DF92EF92FF920F93FD
:101100001F93CF93DF936C017C0187E0E80EF11C05
:10111000D0E0C0E0062F10E0B8010C2E02C075959B
:1011200067950A94E2F76170F70181917F010E944F
:101130009F052196C430D10579F7C601DF91CF9183
:101140001F910F91FF90EF90DF90CF900C94650866
:10115000CF92DF92EF92FF920F931F93CF93DF9383
:10116000EC01F62E642F8C810E949F058D818F3FAC
:1011700019F060E00E949F050F2D10E08F8584FF1D
:1011800025C06E0187E0C80ED11CF12CE12CB801FE
:101190000E2C02C0759567950A94E2F76170F6010E
:1011A00081916F010E949F05FFEFEF1AFF0A88E00F
:1011B000E816F10461F7CE01DF91CF911F910F91F5
:1011C000FF90EF90DF90CF900C946508B80184E019
:1011D000759567958A95E1F7CE010E947B086F2D82
:1011E000CE01DF91CF911F910F91FF90EF90DF9093
:1011F000CF900C947B0840E0682F8AEF96E00C9427
:10120000A808CF93DF93823029F490910907986062
:101210009093090780930D0710920E0780E4809346
:101220000F0780E18093100780E58093110761E04C
:101230008091FE060E94FF058091FF068F3F19F006
:1012400061E00E94FF0561E0809100070E94FF05B8
:10125000CAEFD6E09E012A5F36408091090784FDDF
:101260000BC084E090E021962817390744F461E030
:101270008E810E94FF05EECF88E090E0F4CF8BE3F3
:101280009DE00197F1F760E08091FE060E949F05C6
:1012900060E0809100070E949F058091FF068F3FCC
:1012A00019F060E00E949F058091090784FD39C014
:1012B00063E08AEF96E00E947B08CBE4D6E4CE019F
:1012C0000197F1F763E08AEF96E00E947B0821978F
:1012D000F1F763E08AEF96E00E947B0883E592E0F5
:1012E0000197F1F762E08AEF96E00E947B08809117
:1012F000090780620E94FB0884E080930A078CE063
:101300000E94FB0881E00E94FB088BE39FE10197AC
:10131000F1F782E080930B0786E0DF91CF910C9488
:10132000FB0880620E94FB088BE496E40197F1F7CA
:101330008091090780620E94FB0883E592E0019793
:10134000F1F78091090780620E94FB08D0CF90914D
:101350000D07691710F06FEF690FE62FF0E0E65008
:10136000F94F9489890F80680C94FB0841E00E9432
:10137000A80881E090E008950F931F93CF93DF9327
:101380008B0128E0829FC001112480640E94FB0829
:10139000E801085F1F4F69918AEF96E00E94B60945
:1013A000C017D107C1F7DF91CF911F910F91089519
:1013B00041E0682F8AEF96E00E94A80881E090E063
:1013C0000895FC0101900020E9F73197AF01481B17
:1013D000590BBC018AEF96E00C9437048F929F92D0
:1013E000AF92BF920F931F93CF93DF93CDB7DEB72A
:1013F000A1970FB6F894DEBF0FBECDBF19A2423041
:1014000008F44AE08E010F5D1F4F842E912CB12C01
:10141000A12CA50194010E944533E62FB901CA0110
:10142000EA30F4F4E05DD801EE938D01232B242BF8
:10143000252B79F790E080E0109719F0CD010E94FC
:10144000E109A1960FB6F894DEBF0FBECDBFDF91C4
:10145000CF911F910F91BF90AF909F908F90089563
:10146000E95CE1CFCF92DF92EF92FF92CF93DF93CF
:1014700097FF19C06B017C018DE20E94D809EC0135
:1014800066277727CB016C197D098E099F094AE0F1
:101490000E94EE098C0F9D1FDF91CF91FF90EF907E
:1014A000DF90CF9008954AE0DF91CF91FF90EF90C9
:1014B000DF90CF900C94EE090C94E109CF92DF926B
:1014C000EF92FF92C0902005D0902105E090220578
:1014D000F09023058AE0C816D104E104F1041CF45D
:1014E00080E20E94D80980E20E94D809C701B601B3
:1014F0000E94320A8EE20E94D80960912405709100
:101500002505809126059091270520E432E44FE0DF
:1015100050E00E94673328EE33E040E050E00E9444
:10152000673369017A01C0922005D0922105E092CB
:101530002205F092230584E6C816D104E104F104E3
:1015400064F480E30E94D8098AE0C816D104E1045B
:10155000F1041CF480E30E94D809C701B6010E947F
:10156000320A8EE20E94D809609124057091250507
:10157000809126059091270528EE33E040E050E069
:101580000E9467336B017C01C0922005D092210537
:10159000E0922205F092230584E6C816D104E10406
:1015A000F10464F480E30E94D8098AE0C816D104EB
:1015B000E104F1041CF480E30E94D809C701B601DC
:1015C0000E94320A88E394E0FF90EF90DF90CF9082
:1015D0000C945C0A60E084E00E94A7098091BA0143
:1015E0009091BB01A091BC01B091BD0180932405F5
:1015F00090932505A0932605B09327056091BA0125
:101600007091BB018091BC019091BD0120E432E456
:101610004FE050E00E944533209320053093210590
:1016200040932205509323050E945E0A60E08FE0FC
:101630000E94A70983EB96E00C94640480911C053A
:1016400090911D0561E0019709F451C080E00E946E
:10165000A7098091840190918501A0918601B091A4
:10166000870184369105A105B10591F190F48A3086
:101670009105A105B10531F182339105A105B105AF
:1016800021F10197A105B105C1F580E192E00C942B
:101690005C0A883E23E09207A105B105F9F030F419
:1016A000843F9140A105B105B1F00895803127E252
:1016B0009207A105B105A9F0803A9648A140B1056D
:1016C00099F0089585E192E0E2CF8AE192E0DFCFE0
:1016D0008FE192E0DCCF84E292E0D9CF89E292E020
:1016E000D6CF8EE292E0D3CF83E392E0D0CF80E0FA
:1016F0000E94A70988E392E0CACF0895CF92DF92B3
:10170000EF92FF9261E084E00E94A709C090B601C9
:10171000D090B701E090B801F090B901C701B601CF
:1017200020E432E44FE050E00E946733209320052C
:10173000309321054093220550932305C092240540
:10174000D0922505E0922605F09227050E945E0AB8
:101750008EEB92E0FF90EF90DF90CF900C945C0ABC
:101760004F925F926F927F928F929F92AF92BF92B1
:10177000CF92DF92EF92FF920F931F93CF936B0163
:101780007C01742EAC019B010E941C33882399F0CC
:101790008DE392E0CF911F910F91FF90EF90DF903A
:1017A000CF90BF90AF909F908F907F906F905F9001
:1017B0004F900C94E10946015701E894B7F82FEFD8
:1017C0003FEF4FE75FE7C501B4010E941C33811171
:1017D0000DC02FEF3FEF4FE75FE7C501B4010E9457
:1017E0007E3018161CF481E492E0D4CF2FEF3FEF47
:1017F0004FE75FE4C701B6010E94173318161CF4C7
:1018000085E492E0C7CF2FEF3FEF4FE75FECC701D2
:10181000B6010E947E3087FDF3CF20E030E0A901C1
:10182000C701B6010E947E3010E000E087FF08C0CB
:101830008DE20E94D8098C01F7FAF094F7F8F09441
:10184000C0E060E070E080E09FE37C1641F020E0C3
:1018500030E040E251E40E947632CF5FF6CFA7013C
:1018600096010E940A322B013C010E94E8324B0192
:101870005C014AE00E94EE097C01E00EF11ECC23DF
:10188000B1F1C501B4010E9483309B01AC01C301D9
:10189000B2010E9409324B015C018EE20E94D8091C
:1018A000E80EF91EC15018F120E030E040E251E4AA
:1018B000C501B4010E94E4302B013C010E94E832D2
:1018C0004B01B12CA12C4AE0C501B4010E94EE09E4
:1018D000E80EF91EC501B4010E9483309B01AC01E2
:1018E000C301B2010E9409324B015C01DBCFC70189
:1018F000CF911F910F91FF90EF90DF90CF90BF900D
:10190000AF909F908F907F906F905F904F900895D1
:101910002F923F924F925F926F927F928F929F92FF
:10192000AF92BF92CF92DF92EF92FF920F931F93ED
:10193000CF93DF93CDB7DEB72D970FB6F894DEBF08
:101940000FBECDBF3C01C982DA82EB82FC820D83DF
:101950001E832F83388749875A876B877C878AA1A4
:101960008D873C2C2D2C9E2C502E412EB22EC984BE
:10197000DA84EB84FC8484E190E00E9426358C01BB
:10198000FC01D082C182862D880F880F880F845D6C
:101990000E94C507F92DF3709F2E8C7F982AF801BD
:1019A0009282238234824CE0F694E794D794C794D1
:1019B0004A95D1F7FC2DF07FCF2E8B2D8F70C82A42
:1019C000F801C58246825782B80182E3F1E06F16C2
:1019D000710431F082E06816710409F447C08AE2AC
:1019E0000E947A0730E1F32EF60C8F2D0E94C50776
:1019F00091E0682FA9123CC060648F2D0E9460079F
:101A0000E1E06E167104B1F1F2E06F167104B9F104
:101A1000A092ED062CE2F22E8F2D0E94C50783784E
:101A20009D8591118C60E0E18E9EB0011124682BA0
:101A30008F2D0E946007C8012D960FB6F894DEBF67
:101A40000FBECDBFDF91CF911F910F91FF90EF900F
:101A5000DF90CF90BF90AF909F908F907F906F90CE
:101A60005F904F903F902F900C94C2358AE3B8CF8F
:101A70006F7BC3CFA092EE0694E3F92ECDCFA09258
:101A8000EF068CE3F82EC8CF2F923F924F925F92D1
:101A90006F927F928F929F92AF92BF92CF92DF927E
:101AA000EF92FF920F931F93CF93DF93CDB7DEB7E3
:101AB0006A970FB6F894DEBF0FBECDBF2F8B398764
:101AC000488F598F6A877A8F1C011E8B0D8B60910E
:101AD000F6067091F7068091F8069091F90624E6D3
:101AE00030E040E050E00E94ED33522E632E742E21
:101AF000852E962E788B8F87492E8091F0069091B7
:101B0000F106A091F206B091F3066C017D01FF0C85
:101B1000CC08DC2C76019C01AD016C2D7C2D8C2D2C
:101B20009C2D0FE10E94B834A12CEAECBE2EFAE9FC
:101B3000CF2EABE3DA2EE12CF12C00E010E00E9476
:101B40001A34A52CB62CC72CD82CE92CF8880F8574
:101B5000142D0E9486330FE10E94D33429833A83E7
:101B60004B835C836D837E838F83988789819A8181
:101B7000AB81BC81BB0F880B982FDC018B879C87C6
:101B8000AD87BE87252D362D472D582D692D7F2DEC
:101B90008F85942DA980BA80CB80DC80EB84FE2CCD
:101BA0000E2D1E2D0E94EE3429833B874F87588BC4
:101BB000698B7A8B8B8B9C8B8F889A8C282D39859F
:101BC000488D598D6A85792DC101211534404B46C8
:101BD000544F644171058105910569F060F0812CD5
:101BE000B4E0B987EBE6E88FF4EFF98F84E18A87F8
:101BF000912C212C312C282D3985488D598D6A85C1
:101C0000792DC101211538454744584F6D40710564
:101C10008105910560F4812CB8E5B987E7E4E88F88
:101C2000F8EFF98F8DE08A87912C212C312CA98037
:101C3000BB84CF84D888E988FA880B891C89282D31
:101C40003985488D598D6A85792DC1010E944B34A3
:101C500029013A011FE0A12E9FE0491651046104B9
:101C6000710440F0ABE54A16510461047104D0F0F0
:101C7000BAE5AB2EB12CC12CD12CE12CF12C00E01B
:101C800010E029813B854F85588969897A898B893C
:101C90009C890E948633822E3987488F598F6A87A4
:101CA000972E1C01A980BB84CF84D888E988FA8844
:101CB0000B891C89282D3985488D598D6A85792D88
:101CC000C1010E944934AA24AA94BB24BA94AFE06B
:101CD000CA2ED12CE12CF12C00E010E00E948633BA
:101CE000A980BB84CF84D888E988FA880B891C89AD
:101CF0000E944B34C901DA01812C912C5401839448
:101D00000097A105B10531F088248A94982CEFE062
:101D1000AE2EB12CBC01CD0127E0660F771F881FC6
:101D2000991F2A95D1F7A50194010E944533362EBB
:101D3000272E182F67E0440C551C661C771C6A95EB
:101D4000D1F7B2E05B1A61087108420E531E641E9F
:101D5000751E84E190E00E9426359A838983FC01F8
:101D600090828182862D83708283538244827CE0BC
:101D7000B694A794979487947A95D1F7F82DF07F2D
:101D80008F2E812AA981BA8115968C921597169665
:101D90002C92169717963C921797ED89FE89BD01F4
:101DA0008AE1EF2B19F069817A8182E20E947A0739
:101DB00089819A816A960FB6F894DEBF0FBECDBFB7
:101DC000DF91CF911F910F91FF90EF90DF90CF9017
:101DD000BF90AF909F908F907F906F905F904F904B
:101DE0003F902F900C94C2352F923F924F925F926A
:101DF0006F927F928F929F92AF92BF92CF92DF921B
:101E0000EF92FF920F931F93CF93DF93CDB7DEB77F
:101E1000AA970FB6F894DEBF0FBECDBF622E298FF2
:101E2000732E3A8F4B8F5C8F6D8F7E8F8F8F98A321
:101E300019A708A793012F3F34434C405105610572
:101E400071058105910509F050F4198E85E38A8F9B
:101E50008CE08B8F1C8E1D8E1E8E1F8E18A2298DDE
:101E60003A8D4B8D5C8D6D8D7E8D8F8D98A121155A
:101E7000304A4C4A594B634071058105910569F020
:101E800060F0198E80EA8A8F8CEA8B8F89EB8C8FB9
:101E900083E08D8F1E8E1F8E18A2CE0149960E9460
:101EA000F7028FA3798CBA8DAB8DFC8DED8D6E8C86
:101EB0005F8C48A0272D3B2F4A2F5F2F6E2F762D4A
:101EC000852D942D2F3F05ED300701E140070EE7EA
:101ED000500703E0600771058105910511F008F0D6
:101EE0009EC0CE010D964C01A12CE4E0BE2EFBE677
:101EF000CF2EA4EFDA2EB4E1EB2EF12C00E010E0AF
:101F0000852D942D0E94F300798D6A8D5B8D4C8D0B
:101F10003D8D2E8D9F8D88A1E8A5F9A5E130F105B5
:101F200009F445C0329709F45EC07093D5066093FA
:101F3000D6065093D7064093D8063093D9062093FF
:101F4000DA069093DB068093DC0680E019A2412C30
:101F5000F4E0FAA30BE60BA314EF1CA394E19DA3FA
:101F6000512C612C712C8F938FA0A82ECD84DE84F0
:101F7000EF84F88809891A892B893C894D895E8903
:101F80006F89788D88A599A50E94880C0F9099A1DA
:101F9000913009F0FBC08101242D3AA14BA15CA135
:101FA0006DA1752DC3010E94440D19A2EFC070935D
:101FB000DD066093DE065093DF064093E006309323
:101FC000E1062093E2069093E3068093E40680E026
:101FD00019A2412CE4E0EAA3FBE6FBA304EF0CA367
:101FE00014E11DA3BDCF7093E5066093E606509300
:101FF000E7064093E8063093E9062093EA069093BB
:10200000EB068093EC0680E019A2412C94E09AA3A1
:10201000EBE6EBA3F4EFFCA304E10DA3A1CFCE010B
:102020000D964C01A12CB12CC12CD12CE12CF12C02
:1020300000E010E0852D942D0E94F300298C3A8C4D
:10204000BB8DAC8DFD8DEE8D08A519A50130110558
:1020500009F44EC00230110509F4A5C100E010E0FA
:1020600091014B2F5A2F6F2F7E2F8F8D98A10E9499
:10207000F300422E3AA34BA35CA36DA3572E3C0161
:1020800070E060E090E080E00E9450084092C50659
:102090009AA19093C606EBA1E093C706FCA1F0932A
:1020A000C8060DA10093C9065092CA066092CB06DD
:1020B0007092CC06898D8093D5068A8D8093D60642
:1020C0008B8D8093D7068C8D8093D8068D8D8093D1
:1020D000D9068E8D8093DA068F8D8093DB0688A1DA
:1020E0008093DC0681E011E019A3312C212C3BCF39
:1020F0000F8D09A318A11EA31091F506123009F047
:1021000019C191014B2F5A2F6F2F7E2F802F9EA127
:1021100030584A41564061097109810991092F37A8
:10212000304E42475849624071058105910509F0DA
:1021300008F446C02091E5063091E6064091E70696
:102140005091E8066091E9067091EA068091EB06ED
:102150009091EC065101CB2EDA2EEF2EFE2E09A126
:102160001EA10E94F73461F11092DD061092DE0686
:102170001092DF061092E0061092E1061092E2063D
:102180001092E3061092E40611E019A389A1AA9621
:102190000FB6F894DEBF0FBECDBFDF91CF911F9178
:1021A0000F91FF90EF90DF90CF90BF90AF909F90F6
:1021B0008F907F906F905F904F903F902F900895F9
:1021C0004090CD068091CE068AA39091CF069BA326
:1021D0000091D0060CA31091D1061DA35090D206F9
:1021E0006090D3067090D406CE010D964C01A42CBD
:1021F000BAA0CBA0D02EE12EF52C830191014B2F5C
:102200005A2F6F2F7E2F89A19EA10E94F30061E0BB
:1022100070E081E090E00E94500819A2298D3A8D6B
:102220004B8D5C8D6D8D7E8D8F8D98A130584A4180
:10223000564061097109810991092F37304E424793
:102240005849624071058105910509F008F4A7C05D
:1022500081E08093F5062091E5063091E6064091F5
:10226000E7065091E8066091E9067091EA068091D0
:10227000EB069091EC06A0E00E940035F1F185EEAE
:1022800096E00E94F7028FA3A090CD06B090CE06F4
:10229000C090CF06D090D006E090D106F090D20644
:1022A0000091D3061091D4062091E5063091E60600
:1022B0004091E7065091E8066091E9067091EA06C0
:1022C000CE0101964C018091EB069091EC060E94A4
:1022D000F3001F928FA0A12CC980DA80EB80FC80D4
:1022E0000D811E812F81388549855A856B857C85B6
:1022F00082E090E00E94880C0F90898D8093DD062B
:102300008A8D8093DE068B8D8093DF068C8D809383
:10231000E0068D8D8093E1068E8D8093E2068F8D91
:102320008093E30688A18093E40681E0222423942D
:10233000312C19CE2093CD063093CE064093CF0694
:102340005093D0066093D1067093D2068093D30643
:102350009093D4068E01035F1F4F4801A12CB12C2E
:10236000C12CD12CE12CF12C00E010E091014B2F7D
:102370005A2F6F2F7E2F89A19EA10E94F300422E1B
:102380003AA34BA35CA36DA3572E3C0161E070E020
:1023900081E090E00E94500811E019A33FCF88E04F
:1023A0008093F506AACF0091F50609A31F8D1EA301
:1023B00008A10AA719A1113009F0F9C091014B2F0A
:1023C0005A2F6F2F7E2F8EA1902F30584A415640A2
:1023D00061097109810991092F37304E42475849E7
:1023E000624071058105910561F158F12091E50682
:1023F0003091E6064091E7065091E8066091E906C3
:102400007091EA068091EB069091EC065101CB2E7B
:10241000DA2EEF2EFE2E0EA11AA50E94F73489F0B7
:102420001092E5061092E6061092E7061092E80672
:102430001092E9061092EA061092EB061092EC0652
:10244000A5CE4090CD061091CE061AA38091CF065E
:102450008BA39091D0069CA30091D1060DA3509020
:10246000D2066090D3067090D406CE010D964C0132
:10247000A42CB12ECBA0DCA0E02EF52C8301910181
:102480004B2F5A2F6F2F7E2F8EA19AA50E94F300FB
:1024900061E070E082E090E00E94500819A2298D6E
:1024A0003A8D4B8D5C8D6D8D7E8D8F8D98A13058C2
:1024B0004A41564061097109810991092F37304E0F
:1024C00042475849624071058105910509F008F4B9
:1024D000A3C082E08093F5062091DD063091DE06F0
:1024E0004091DF065091E0066091E1067091E206AE
:1024F0008091E3069091E406A0E00E940035F1F19E
:102500008DED96E00E94F7028FA3A090CD06B090CB
:10251000CE06C090CF06D090D006E090D106F090C5
:10252000D2060091D3061091D4062091DD06309199
:10253000DE064091DF065091E0066091E106709161
:10254000E206CE0101964C018091E3069091E406EB
:102550000E94F3001F928FA0A12CC980DA80EB802B
:10256000FC800D811E812F81388549855A856B85B8
:102570007C8581E090E00E94880C0F90898D80938B
:10258000E5068A8D8093E6068B8D8093E7068C8D19
:102590008093E8068D8D8093E9068E8D8093EA0600
:1025A0008F8D8093EB0688A18093EC06BECE20939E
:1025B000CD063093CE064093CF065093D00660935D
:1025C000D1067093D2068093D3069093D4068E01E1
:1025D000035F1F4F4801A12CB12CC12CD12CE12C41
:1025E000F12C00E010E091014B2F5A2F6F2F7E2F1E
:1025F0008EA19AA50E94F300422E3AA34BA35CA39E
:102600006DA3572E3C0161E070E082E090E00E94F3
:10261000500811E019A343CF88E08093F506AECFB0
:10262000CF93DF93EC0188819981009711F00E948C
:10263000C235198218821D821C821B821A82DF9188
:10264000CF910895FC01808191810C94C2350F9344
:102650001F93CF93DF938C01EB010E94A2318883FB
:10266000C80101960E94A2318983CE01DF91CF91EA
:102670001F910F910895CF92DF92EF92FF920F93E7
:102680001F93CF93DF93EB017B0124E0E20EF11C5B
:102690008B016C01C61AD70AC601800F911F0E94D8
:1026A000A231F80181938F01EE15FF05A9F7CE0144
:1026B000DF91CF911F910F91FF90EF90DF90CF901E
:1026C0000895CF93DF93C0911605D091170568E266
:1026D00071E08AEA90E0209739F0C130D105E1F548
:1026E00064E271E08FEA90E00E943B13FC0180817C
:1026F0009181A281B3818093BA019093BB01A09391
:10270000BC01B093BD0110923005109231051092BA
:1027100032051092330564E171E083EC90E0C5303E
:10272000D105C1F50E943B13FC0180819181A281FA
:10273000B3818093BA019093BB01A093BC01B09385
:10274000BD011092300510923105109232051092A1
:102750003305DF91CF910895C230D10519F560E2BC
:1027600071E084EB90E00E943B13FC018081918139
:10277000A281B3818093BA019093BB01A093BC0165
:10278000B093BD01109230051092310510923205C0
:102790001092330560E171E088EC90E0C630D1051D
:1027A00009F21EC0C330D10561F56CE171E089EB1F
:1027B00090E00E943B13FC0180819181A281B38152
:1027C0008093BA019093BB01A093BC01B093BD016B
:1027D0001092300510923105109232051092330597
:1027E0006CE071E08DEC90E0C730D10509F49ACF30
:1027F00068E071E082ED90E0C830D10509F492CF35
:102800001FC0C430D10509F086CF68E171E08EEBBE
:1028100090E00E943B13FC0180819181A281B381F1
:102820008093BA019093BB01A093BC01B093BD010A
:102830001092300510923105109232051092330536
:10284000299709F086CF64E071E087ED90E06ACFC8
:10285000CF93DF93EB010E94A2318883CE01DF91F9
:10286000CF9108950F931F93CF93DF93EC0188814D
:102870009981009759F02A813B812617370730F05C
:1028800081E0DF91CF911F910F9108958B016F5FD0
:102890007F4F0E944B36009759F0998388831B83A2
:1028A0000A832C813D81232B59F7FC011082E8CF4C
:1028B00080E0E7CFEF92FF920F931F93CF93DF93C8
:1028C0006115710541F480E0DF91CF911F910F9167
:1028D000FF90EF90089541155105B1F07B01EC0197
:1028E0000C811D81040F151FB8010E94321488232A
:1028F00051F3288139818C819D81B701820F931F0B
:102900000E941A371D830C8381E0DECFFC01019009
:102910000020E9F73197AF01481B590BBC018BE947
:1029200096E00C945A14EF92FF920F931F93CF935B
:10293000DF93EC017B018A01BA010E9432148111FC
:102940000BC0CE010E941013CE01DF91CF911F91D9
:102950000F91FF90EF9008951D830C83B70188813C
:1029600099810E941A37F0CFFB0101900020E9F70E
:102970003197AF01461B570B0C949314FC01118245
:1029800010821382128215821482FB0101900020B2
:10299000E9F73197AF01461B570B0C949314FF9244
:1029A0000F931F93CF93DF93EC01F62E08811981CB
:1029B000C8010E94A231F81621F06F2DC8010E94B3
:1029C000AA31CE01DF91CF911F910F91FF90089511
:1029D000EF92FF920F931F93CF93DF9300D0CDB769
:1029E000DEB70AEB11E08A5B91407C01C701800FE2
:1029F000911F9A838983F80161918F01CE0101961D
:102A00000E94CF14F1E00E3B1F0781F78AEB91E0A3
:102A10000F900F90DF91CF911F910F91FF90EF904A
:102A200008954091BA015091BB016091BC01709131
:102A3000BD018091520590915305A0915405B0912C
:102A40005505481759076A077B0709F4BFC08091ED
:102A5000BA019091BB01A091BC01B091BD01803140
:102A60009742A105B105B8F08091BA019091BB01E0
:102A7000A091BC01B091BD01803C964CAD42B10526
:102A800050F415B810921705109216058AEA90E0D6
:102A90000E94E8148BC08091BA019091BB01A09173
:102AA000BC01B091BD01803C964CAD42B10570F0C7
:102AB0008091BA019091BB01A091BC01B091BD0180
:102AC00080349B44AC44B10508F481C08091BA01C4
:102AD0009091BB01A091BC01B091BD0180349B4499
:102AE000AC44B10508F07EC08091BA019091BB0161
:102AF000A091BC01B091BD0181159241AA47B105D9
:102B000008F089C08091BA019091BB01A091BC01ED
:102B1000B091BD0181159B41A74BB10508F094C050
:102B20008091BA019091BB01A091BC01B091BD010F
:102B300081159442A44FB10508F09FC08091BA015D
:102B40009091BB01A091BC01B091BD01803C9A4E17
:102B5000A142B14008F0AAC08091BA019091BB0196
:102B6000A091BC01B091BD018038914BAF44B14000
:102B700008F0B5C08091BA019091BB01A091BC0151
:102B8000B091BD01803C9C4FAB49B14008F0C0C042
:102B90008091BA019091BB01A091BC01B091BD019F
:102BA00081159A45A246B24008F0CBC08091BA0187
:102BB0009091BB01A091BC01B091BD0180935205E1
:102BC00090935305A0935405B0935505089584E060
:102BD00085B981E090E090931705809316058FEA00
:102BE00090E056CF8091BA019091BB01A091BC01B9
:102BF000B091BD0181159241AA47B10508F074CF8B
:102C000088E085B982E090E09093170580931605DF
:102C100084EB90E03DCF8091BA019091BB01A091EF
:102C2000BC01B091BD0181159B41A74BB10508F0D6
:102C300069CF8CE085B983E090E09093170580938D
:102C4000160589EB90E024CF8091BA019091BB01E9
:102C5000A091BC01B091BD0181159442A44FB10572
:102C600008F05ECF80E185B984E090E0909317058D
:102C7000809316058EEB90E00BCF8091BA01909176
:102C8000BB01A091BC01B091BD01803C9A4EA14214
:102C9000B14008F053CF84E185B985E090E090938E
:102CA00017058093160583EC90E0F2CE8091BA016F
:102CB0009091BB01A091BC01B091BD018038914BB6
:102CC000AF44B14008F048CF88E185B986E090E094
:102CD000909317058093160588EC90E0D9CE8091EB
:102CE000BA019091BB01A091BC01B091BD01803CA3
:102CF0009C4FAB49B14008F03DCF8CE185B987E0EE
:102D000090E090931705809316058DEC90E0C0CE6F
:102D10008091BA019091BB01A091BC01B091BD011D
:102D200081159A45A246B24008F032CF80E285B9BB
:102D300088E090E0909317058093160582ED90E06F
:102D4000A7CE8091BA019091BB01A091BC01B09136
:102D5000BD018130924CAB4EBB4008F027CF84E2DE
:102D600085B989E090E0909317058093160587ED6B
:102D700090E08ECEAF92BF92CF92DF92EF92FF9211
:102D80000F931F93CF93DF9300D0CDB7DEB78B01A6
:102D90006B0124E0C20ED11C7B015C01A61AB70AAC
:102DA000C5018E0D9F1D9A838983F70161917F0173
:102DB000CE0101960E94CF14EC14FD0489F7C801DE
:102DC0000F900F90DF91CF911F910F91FF90EF9097
:102DD000DF90CF90BF90AF900895EF92FF920F9346
:102DE0001F93CF93DF9300D0CDB7DEB78C017B016B
:102DF0009A838983FB016081CE0101960E94CF14E2
:102E00000F5F1F4F1A830983F7016181CE0101967D
:102E10000E94CF14C7010F900F90DF91CF911F91A7
:102E20000F91FF90EF9008950F931F93CF93DF932F
:102E30008091670590916805019701F560E080E059
:102E40000E94A70989E492E00E945C0A0E941E0B7E
:102E500061E084E00E94A70987E394E00E945C0A95
:102E60006091340170913501809136019091370164
:102E70000E94320A86E694E00E945C0A809167050F
:102E800090916805029761F40E947E0B60E080E0FB
:102E90000E94A7098BE592E00E945C0A0E941E0B2B
:102EA0008091670590916805039749F50E947E0B14
:102EB00060E080E00E94A7098CE692E00E945C0A34
:102EC00080915A05811106C06DE772E089E896E0AD
:102ED0000E94B41480915A05813031F461E872E0A7
:102EE00089E896E00E94B41461E080E00E94A7099E
:102EF00089E896E00E94640480E20E94D8098091EB
:102F0000670590916805049721F50E94EA0A80916F
:102F10006305811106C06DE772E08FE896E00E94BC
:102F2000B41480916305813031F461E872E08FE878
:102F300096E00E94B41461E080E00E94A7098FE847
:102F400096E00E94640485E892E00E945C0A0E9478
:102F5000EA0A8091670590916805059701F560E0A0
:102F600080E00E94A70983E992E00E945C0A0E9427
:102F70001E0B61E084E00E94A70987E394E00E94B1
:102F80005C0A60914E0570914F05809150059091BB
:102F900051050E94320A84EA92E00E945C0A809104
:102FA000670590916805069709F560E080E00E944A
:102FB000A7098CEA92E00E945C0A61E080E00E942E
:102FC000A70982E494E00E945C0A6091300170914C
:102FD000310180913201909133010E94320A8DEBD0
:102FE00092E00E945C0A80E20E94D8098091670505
:102FF000909168050797C1F460E080E00E94A709FE
:1030000081EC92E00E945C0A61E080E00E94A709E6
:1030100086E694E00E945C0A83E896E00E946404DD
:103020008EE494E00E945C0A8091670590916805A7
:10303000089709F01AC28091870690918806892B1B
:1030400009F413C2C0918306D09184066DE772E043
:10305000CE010E941137892B21F41092680510923D
:10306000670561E872E0CE010E941137892B09F0F3
:10307000F2C10E94A40600914005109141052091E3
:10308000420530914305601B710B820B930B653F2A
:1030900071408105910508F4DEC161E080E00E9485
:1030A000A70982ED92E00E945C0A6091B6047091DB
:1030B000B7048091B8049091B90442E00E94B00B2B
:1030C00083E493E00E945C0A80910F058130C1F493
:1030D0000E94A30760E080E00E94A7098EED92E0C5
:1030E0000E945C0A80913E0590913F0590932F01CC
:1030F00080932E016EE271E084E690E00E94ED166E
:1031000080910F058230D1F50E94A30760E080E036
:103110000E94A70980EF92E00E945C0A80913E0520
:1031200090913F0590938D0180938C0120912E0109
:1031300030912F01821B930B63E070E00E943133CA
:10314000260F371F30932D0120932C01260F371F98
:1031500030938B0120938A016CE271E087E690E066
:103160000E94ED166AE871E08AE690E00E94ED1692
:103170006CE871E08DE690E00E94ED1680910F05FD
:103180008330D1F50E94A30760E080E00E94A70988
:1031900081E093E00E945C0A80913E0590913F059A
:1031A000909393018093920120918C0130918D0135
:1031B000821B930B63E070E00E943133260F371FB0
:1031C00030938F0120938E01260F371F309391018A
:1031D000209390016EE871E080E790E00E94ED1688
:1031E00060E971E083E790E00E94ED1662E971E02A
:1031F00086E790E00E94ED1680910F058430D1F5AE
:103200000E94A30760E080E00E94A70982E193E0AA
:103210000E945C0A80913E0590913F059093990130
:10322000809398012091920130919301821B930B1E
:1032300063E070E00E943133260F371F3093950111
:1032400020939401260F371F309397012093960106
:1032500064E971E089E790E00E94ED1666E971E0AB
:103260008CE790E00E94ED1668E971E08FE790E04E
:103270000E94ED1680910F05853009F048C00E942C
:10328000A30760E080E00E94A70983E293E00E9428
:103290005C0A80913E0590913F059093A101809337
:1032A000A0012091980130919901821B930B97FD09
:1032B00003969595879595958795280F391F309397
:1032C0009B0120939A01280F391F30939D01209371
:1032D0009C01820F931F90939F0180939E016AE946
:1032E00071E082E890E00E94ED166CE971E085E8FB
:1032F00090E00E94ED166EE971E088E890E00E948F
:10330000ED1660EA71E08BE890E00E94ED16809186
:103310000F05863009F048C00E94A30760E080E0F6
:103320000E94A70984E393E00E945C0A80913E0515
:1033300090913F059093A9018093A8012091A0014D
:103340003091A101821B930B97FD0396959587956C
:1033500095958795280F391F3093A3012093A201DB
:10336000280F391F3093A5012093A401820F931FCA
:103370009093A7018093A60162EA71E08EE890E045
:103380000E94ED1664EA71E081E990E00E94ED167A
:1033900066EA71E084E990E00E94ED1668EA71E067
:1033A00087E990E00E94ED1680910F05873009F0C3
:1033B00048C00E94A30760E080E00E94A70985E45E
:1033C00093E00E945C0A80913E0590913F059093A6
:1033D000B1018093B0012091A8013091A901821B15
:1033E000930B97FD03969595879595958795280F4F
:1033F000391F3093AB012093AA01280F391F309356
:10340000AD012093AC01820F931F9093AF01809385
:10341000AE016AEA71E08AE990E00E94ED166CEA7A
:1034200071E08DE990E00E94ED166EEA71E080EAAD
:1034300090E00E94ED1660EB71E083EA90E00E945C
:10344000ED160E94A4066093400570934105809399
:10345000420590934305809167059091680509970F
:1034600024F01092680510926705DF91CF911F91AB
:103470000F910C9411150F931F93CF93DF9300D0EE
:10348000CDB7DEB78B019A838983FB016081CE01C2
:1034900001960E94CF14C8010F900F90DF91CF9139
:1034A0001F910F9108958F929F92AF92BF92FF92BA
:1034B0000F931F93CF93DF93EC01F090650500917C
:1034C000670510916805F11052C00230110509F42A
:1034D0004EC08130910509F0B6C080910F058F5F15
:1034E000873008F0AEC080930F0540918401509161
:1034F000850160918601709187018091BA01909158
:10350000BB01A091BC01B091BD01840F951FA61F06
:10351000B71F8093BA019093BB01A093BC01B093F5
:10352000BD016091BA017091BB018091BC01909185
:10353000BD01209184013091850140918601509117
:1035400087018090840190908501A0908601B090C1
:1035500087010E944533C501B4010E942133609365
:10356000BA017093BB018093BC019093BD0180911F
:10357000BA019091BB01A091BC01B091BD0181380D
:10358000944AAF4BB74060F080E894EAAFEBB7E005
:103590008093BA019093BB01A093BC01B093BD018D
:1035A0008091BA019091BB01A091BC01B091BD0185
:1035B000803A9648A140B10560F480EA96E8A1E01F
:1035C000B0E08093BA019093BB01A093BC01B0938B
:1035D000BD0181E0F812BBC0C130D10509F082C045
:1035E000409184015091850160918601709187011D
:1035F0008091300590913105A0913205B09133054D
:10360000840F951FA61FB71F809330059093310537
:10361000A0933205B09333050130110509F0D0C0F5
:103620008091520590915305A0915405B091550594
:103630008093BA019093BB01A093BC01B093BD01EC
:103640009DC087E050CF019609F091CF4091840151
:103650005091850160918601709187018091BA0136
:103660009091BB01A091BC01B091BD01841B950B51
:10367000A60BB70B8093BA019093BB01A093BC013A
:10368000B093BD016091BA017091BB018091BC0102
:103690009091BD0120918401309185014091860176
:1036A000509187018090840190908501A0908601BF
:1036B000B09087010E944533C501B4010E942133B7
:1036C0006093BA017093BB018093BC019093BD01DC
:1036D00080910F058150823018F080930F0547CFFD
:1036E00081E0FBCFCF3FDC0709F031C2409184017C
:1036F000509185016091860170918701809130051C
:1037000090913105A0913205B0913305841B950B42
:10371000A60BB70B8093300590933105A09332052B
:10372000B09333050130110509F04AC0809152056C
:1037300090915305A0915405B09155058093BA011D
:103740009093BB01A093BC01B093BD0179C101303E
:103750001105B1F58091520590915305A091540542
:10376000B09155058093BA019093BB01A093BC0121
:10377000B093BD01C130D10509F05EC14091840113
:10378000509185016091860170918701809134018B
:1037900090913501A0913601B0913701840F951FAA
:1037A000A61FB71F8093340190933501A093360173
:1037B000B093370164E371E08AE190E00E94BA16A9
:1037C00080916705909168050297E1F58091520517
:1037D00090915305A0915405B09155058093BA017D
:1037E0009093BB01A093BC01B093BD01CF3FDC0718
:1037F00019F58091B6019091B701A091B801B091EF
:10380000B901813A26E8920721E0A207B105A4F0A8
:1038100040918401509185016091860170918701EA
:10382000841B950BA60BB70B8093B6019093B70141
:10383000A093B801B093B90166EB71E085E190E027
:103840000E94BA168091670590916805039719F553
:103850008091520590915305A0915405B091550562
:103860008093BA019093BB01A093BC01B093BD01BA
:10387000C130D10509F0F9C061E872E089E896E04D
:103880000E94B41481E080935A056AE575E08DE0EA
:1038900090E00E943B1A809167059091680504971B
:1038A00019F58091520590915305A0915405B0915E
:1038B00055058093BA019093BB01A093BC01B093CE
:1038C000BD01C130D10509F0DDC061E872E08FE8CB
:1038D00096E00E94B41481E08093630563E675E08E
:1038E00090E080E00E943B1A809167059091680506
:1038F0000597B1F58091520590915305A09154051B
:10390000B09155058093BA019093BB01A093BC017F
:10391000B093BD01C130D10509F0C1C0409184010F
:1039200050918501609186017091870180914E05CB
:1039300090914F05A0915005B0915105840F951FAE
:10394000A61FB71F80934E0590934F05A093500577
:10395000B09351056EE475E084E290E00E94BA16DF
:1039600080916705909168050697B9F58091520599
:1039700090915305A0915405B09155058093BA01DB
:103980009093BB01A093BC01B093BD01C130D105A0
:1039900009F0A3C08091300190913101A0913201D2
:1039A000B0913301805F984DAF4FBF4F803823EC0B
:1039B000920729ECA20721E0B2070CF089C080939E
:1039C000300190933101A0933201B093330160E351
:1039D00071E088E290E00E94BA16809167059091AC
:1039E00068058730910509F096C080915205909145
:1039F0005305A0915405B09155058093BA01909359
:103A0000BB01A093BC01B093BD016DE772E0CF3F55
:103A1000DC0729F0219709F090C061E872E083E8A3
:103A200096E0DF91CF911F910F91FF90BF90AF90E3
:103A30009F908F900C94B414CF3FDC0709F0BACE5E
:103A400040918401509185016091860170918701B8
:103A50008091340190913501A0913601B0913701E8
:103A6000841B950BA60BB70B9DCECF3FDC0709F04F
:103A70000CCF6DE772E089E896E00E94B4141092D2
:103A80005A0503CFCF3FDC0709F028CF6DE772E07E
:103A90008FE896E00E94B414109263051FCFCF3FC9
:103AA000DC0709F057CF4091840150918501609166
:103AB00086017091870180914E0590914F05A091EC
:103AC0005005B0915105841B950BA60BB70B3ACF4F
:103AD00080E893ECA9ECB1E072CFCF3FDC0709F0AE
:103AE00076CF8091300190913101A0913201B09157
:103AF000330180519742A109B109813026E3920731
:103B00002EE6A20721E0B2070CF059CF80E096E341
:103B1000AEE6B1E054CF089781F4809152059091C0
:103B20005305A0915405B09155058093BA01909327
:103B3000BB01A093BC01B093BD01DF91CF911F9158
:103B40000F91FF90BF90AF909F908F90089501309C
:103B5000110509F035CE8091520590915305A09141
:103B60005405B09155058093BA019093BB01A09381
:103B7000BC01B093BD011ECE1F920F920FB60F92E3
:103B800011242F933F934F935F936F937F938F9362
:103B90009F93AF93BF93EF93FF938AED95E00E94BD
:103BA000BE04FF91EF91BF91AF919F918F917F9153
:103BB0006F915F914F913F912F910F900FBE0F909A
:103BC0001F9018951F920F920FB60F9211242F93EA
:103BD0008F939F93EF93FF93E091EA05F091EB05AC
:103BE0008081E091F005F091F10582FD1BC090818C
:103BF0008091F3058F5F8F732091F405821741F058
:103C0000E091F305F0E0E652FA4F958F8093F305CB
:103C1000FF91EF919F918F912F910F900FBE0F9079
:103C20001F9018958081F4CF1F920F920FB60F92BC
:103C300011242F933F938F939F93AF93BF938091C2
:103C4000FE049091FF04A0910005B0910105309110
:103C5000FD0423E0230F2D3758F50196A11DB11D5A
:103C60002093FD048093FE049093FF04A09300052D
:103C7000B09301058091020590910305A091040580
:103C8000B09105050196A11DB11D80930205909389
:103C90000305A0930405B0930505BF91AF919F91D3
:103CA0008F913F912F910F900FBE0F901F901895FD
:103CB00026E8230F0296A11DB11DD2CF1F920F92AD
:103CC0000FB60F9211242F933F934F935F936F93EF
:103CD0007F938F939F93AF93BF93EF93FF938091C5
:103CE000B900887F803609F44AC0F0F5883209F4BB
:103CF000A7C018F5803109F49BC0B8F4882309F4F3
:103D0000F9C0883009F494C0FF91EF91BF91AF9151
:103D10009F918F917F916F915F914F913F912F91E3
:103D20000F900FBE0F901F901895883109F488C02E
:103D3000803251F78093B30514C0803409F49DC0DC
:103D400040F48033B9F38833F9F68093B30585ECFA
:103D5000B0C0803509F485C0883509F496C0883430
:103D600099F60E94B006D0CF883909F48CC038F596
:103D7000883729F050F4883611F0803729F683E02F
:103D80008093B5051092FC0457C0883809F47BC0B5
:103D9000803919F0803809F0B7CF8091FC04803267
:103DA00008F071C0E091FC0481E08E0F8093FC0468
:103DB0008091BB00F0E0E452FB4F80833DC0803B2C
:103DC00039F0E0F4803A09F479C0883A09F09CCFE0
:103DD00084E08093B5051092DB041092DA04E09140
:103DE0006B05F0916C0509958091DA0481110FC083
:103DF00081E08093DA041092BA0409C0803C09F48F
:103E0000A6CF883C09F4A3CF883B09F07DCFE09191
:103E1000DB0481E08E0F8093DB04F0E0E654FB4F7F
:103E200080818093BB009091DB048091DA0429C0EB
:103E3000809190058093BB0085EC8093BC0064CF9B
:103E40009091B2058091B105981758F5E091B205AF
:103E500081E08E0F8093B205F0E0EF56FA4F80813B
:103E6000E9CFE091B20581E08E0F8093B205809199
:103E7000BB00F0E0EF56FA4F80839091B20580913D
:103E8000B1059817C8F285E8D8CFE091B20581E076
:103E90008E0F8093B2058091BB00F0E0EF56FA4F91
:103EA00080838091B40581115CCF81E080938F0580
:103EB00084EA8093BC001092B50526CF85EC8093F0
:103EC000BC001092B5058091FC04803230F4E09182
:103ED000FC04F0E0E452FB4F10826091FC0470E0BF
:103EE000E0916905F0916A058CED94E009951092D6
:103EF000FC040ACF1092B30534CF1F920F920FB675
:103F00000F921124CF92DF92EF92FF920F931F93A3
:103F10002F933F934F935F936F937F938F939F93D1
:103F2000AF93BF93CF93DF93EF93FF938091BB0643
:103F30000E947605EC018091BA060E947605909168
:103F4000B9069F70CC0FDD1FC82B24E0929FC001E3
:103F500011248C539E4FC80FD92FD11DC881C093F7
:103F6000B906C07361F10E94A40600910605109184
:103F7000070520910805309109056B017C01C01AE5
:103F8000D10AE20AF30A9701860100930B05109308
:103F90000C0520930D0530930E0560930605709374
:103FA0000705809308059093090581E090E0C031F2
:103FB00021F0C03221F48FEF9FEF0E94531AFF913E
:103FC000EF91DF91CF91BF91AF919F918F917F91B1
:103FD0006F915F914F913F912F911F910F91FF90A2
:103FE000EF90DF90CF900F900FBE0F901F9018951D
:103FF000CF93DF93EAEDF5E01382128288EE93E02F
:10400000A0E0B0E084839583A683B78324EE31E0FB
:104010003183208325EC30E03587248724EC30E0A1
:104020003787268720EC30E0318B208B21EC30E085
:10403000338B228B22EC30E0358B248B26EC30E066
:10404000378B268B118E128E138E148EE7E7F6E0D7
:104050001382128284839583A683B78386EF91E0CF
:1040600091838083EAEFF6E01382128288E092E087
:104070009183808389E084838FEF8583C8E0C68342
:1040800087E0878386E0808785E0818784E0828778
:104090001386148615861686178681E00E9401090C
:1040A000ECEBF6E0C0AFC1AF11AA12AA13AA1186B9
:1040B000128613861486158616861786108A118A2C
:1040C000128A138A148A158A168A178A108E118EFC
:1040D000128E138E148E158E168E178E10A211A2AC
:1040E00012A213A214A215A216A217A210A611A61C
:1040F00012A613A614A615A616A617A610AA80ED3A
:1041000090E9A7EFB1E082AF93AFA4AFB5AFC9EB31
:10411000D6E083E0898382E08A8360E083E00E94C6
:10412000FF0560E08A810E94FF0561E089810E94AD
:104130009F0561E08A810E949F05188266E573E011
:1041400083EB96E00E94BE1468E573E08DEA96E08A
:104150000E94BE146DE573E087EA96E00E94BE14EB
:1041600069E374E081EA96E00E94BE1469E374E0BA
:104170008BE996E00E94BE1469E374E085E996E05D
:104180000E94BE146DE772E08FE896E00E94BE14B4
:104190006DE772E089E896E00E94BE146DE772E078
:1041A00083E896E0DF91CF910C94BE14CF93DF9318
:1041B000CDB7DEB7A7970FB6F894DEBF0FBECDBF61
:1041C000789484B5826084BD84B5816084BD85B5F2
:1041D000826085BD85B5816085BD80916E008160FE
:1041E00080936E00109281008091810082608093A4
:1041F00081008091810081608093810080918000A6
:104200008160809380008091B10084608093B100D0
:104210008091B00081608093B00080917A008460CA
:1042200080937A0080917A00826080937A008091F6
:104230007A00816080937A0080917A008068809310
:104240007A001092C100E091EA05F091EB0582E05E
:104250008083E091E605F091E7051082E091E805A2
:10426000F091E9058FEC80831092F205E091EE0564
:10427000F091EF0586E08083E091EC05F091ED058B
:10428000808180618083E091EC05F091ED05808173
:1042900088608083E091EC05F091ED058081806875
:1042A0008083E091EC05F091ED0580818F7D808326
:1042B00082E00E94010981E00E94FB088BE39FE1FC
:1042C0000197F1F70E94CD0561E08AE00E94FF05A9
:1042D00061E08BE00E94FF0561E08CE00E94FF0539
:1042E00061E08DE00E94FF0560E08FE00E94FF0525
:1042F00061E080E10E94FF0561E081E10E94FF052D
:1043000068E671E081E00E94BC0960E671E082E04D
:104310000E94BC0968E571E083E00E94BC0960E589
:1043200071E084E00E94BC0968E471E085E00E94CD
:10433000BC0960E471E086E00E94BC0968E371E0BA
:1043400087E00E94BC096AE075E089E090E00E9485
:104350002814DC018C918F3609F464C763E675E09C
:1043600090E080E00E943B1A65E175E088E090E013
:104370000E943B1A8FE690E09A838983BE016F5FAB
:104380007F4F89E090E00E94ED166AE575E08DE0D0
:1043900090E00E943B1A60E375E08FE090E00E949D
:1043A000BA1666EB71E085E190E00E94BA1664E30C
:1043B00071E08AE190E00E94BA168FE190E00E94DD
:1043C000E8146AE475E084E290E00E94BA1660E3C3
:1043D00071E088E290E00E94BA1668E871E087E335
:1043E00090E00E94ED1660E871E08CE390E00E949E
:1043F000BA166CE771E081E490E00E94BA1668E7B3
:1044000071E086E490E00E94BA1664E771E08BE404
:1044100090E00E94BA1660E771E080E590E00E94AB
:10442000BA166EE271E084E690E00E94ED166CE24E
:1044300071E087E690E00E94ED166AE871E08AE696
:1044400090E00E94ED166CE871E08DE690E00E942D
:10445000ED166EE871E080E790E00E94ED1660E9ED
:1044600071E083E790E00E94ED1662E971E086E773
:1044700090E00E94ED1664E971E089E790E00E9407
:10448000ED1666E971E08CE790E00E94ED1668E9B0
:1044900071E08FE790E00E94ED166AE971E082E832
:1044A00090E00E94ED166CE971E085E890E00E94D2
:1044B000ED166EE971E088E890E00E94ED1660EA82
:1044C00071E08BE890E00E94ED1662EA71E08EE800
:1044D00090E00E94ED1664EA71E081E990E00E94AC
:1044E000ED1666EA71E084E990E00E94ED1668EA54
:1044F00071E087E990E00E94ED166AEA71E08AE9CE
:1045000090E00E94ED166CEA71E08DE990E00E9467
:10451000ED166EEA71E080EA90E00E94ED1660EB25
:1045200071E083EA90E00E94ED1668E271E08AEAA9
:1045300090E00E94BA1664E271E08FEA90E00E9477
:10454000BA1660E271E084EB90E00E94BA166CE16A
:1045500071E089EB90E00E94BA1668E171E08EEBA1
:1045600090E00E94BA1664E171E083EC90E00E9452
:10457000BA1660E171E088EC90E00E94BA166CE037
:1045800071E08DEC90E00E94BA1668E071E082ED77
:1045900090E00E94BA1664E071E087ED90E00E941E
:1045A000BA1663E675E090E080E00E942814DC0112
:1045B0008C918093630565E175E088E090E00E944E
:1045C0002814FC0180818093150566E475E085E17F
:1045D00090E00E943B13FC0180819181A281B38114
:1045E0008093B6019093B701A093B801B093B9013D
:1045F0006AE575E08DE090E00E942814DC018C9162
:1046000080935A0560E375E08FE090E00E943B13D1
:10461000FC0180819181A281B381809330059093C8
:104620003105A0933205B093330564E371E08AE16C
:1046300090E00E943B13FC0180819181A281B381B3
:104640008093340190933501A0933601B0933701E4
:104650008FE190E00E94A2318093000180E290E01F
:104660000E94A2318093010181E290E00E94A23178
:104670008093020182E290E00E94A23180930301C4
:104680008091000190910101A0910201B09103017C
:104690008093BA019093BB01A093BC01B093BD017C
:1046A0006EE475E084E290E00E943B13FC0180819F
:1046B0009181A281B38180934A0590934B05A09389
:1046C0004C05B0934D0560E371E088E290E00E94F4
:1046D0003B13FC0180819181A281B38180933001E1
:1046E00090933101A0933201B093330168E871E0F7
:1046F00087E390E00E942713DC018D919C919093B9
:1047000089018093880160E871E08CE390E00E9469
:104710003B13FC0180819181A281B3818093800150
:1047200090938101A0938201B09383016CE771E0C3
:1047300081E490E00E943B13FC0180819181A28181
:10474000B38180937C0190937D01A0937E01B0930F
:104750007F0168E771E086E490E00E943B13FC0172
:1047600080819181A281B3818093780190937901B6
:10477000A0937A01B0937B0164E771E08BE490E051
:104780000E943B13FC0180819181A281B3818093BF
:10479000740190937501A0937601B093770160E75F
:1047A00071E080E590E00E943B13FC0180819181E3
:1047B000A281B3818093700190937101A0937201E3
:1047C000B09373018091340190913501A09136012D
:1047D000B09137018093F0069093F106A093F20612
:1047E000B093F306C0903001D0903101E0903201D7
:1047F000F09033010E94CD0562E987EB0E946007CB
:10480000C114D104E104F104D1F08FE00E94C50786
:10481000682F6F73F1E8CF16F3ECDF06F9ECEF06C3
:10482000F1E0FF0608F00DC5C092F606D092F7063B
:10483000E092F806F092F9068FE00E94600760E8C7
:1048400080E10E94600760E881E10E94600760E803
:1048500082E10E9460076CE080E10E9460076CE0EA
:1048600081E10E9460076CE082E10E94600760E2E3
:1048700081EB0E94600760E881EB0E94600710E016
:1048800000E020E034E04BE654EF64E170E080E0CB
:1048900090E00E94440D61E081E090E00E943808C1
:1048A00090E080E00E942C0881E090E00E942C08BB
:1048B00082E090E00E942C0866E573E083EB96E0CE
:1048C0000E94B41462E08EE00E94FF0580916800AF
:1048D00084608093680080916D008C6080936D008F
:1048E00078940E94A4066093060570930705809350
:1048F00008059093090588EE93E0A0E0B0E080936E
:104900000B0590930C05A0930D05B0930E05109127
:104910001505113061F461E673E08DEA96E00E94BE
:10492000B4141093440561E080E10E949F058091DA
:10493000150581110CC068E573E08DEA96E00E94D0
:10494000B4141092440560E080E10E949F059091AC
:104950001905809164059111AAC4883208F07DC0C0
:10496000809114058130A9F460E871E08CE390E057
:104970000E943B13FC0180819181A281B3818093CD
:10498000BA019093BB01A093BC01B093BD011092FA
:104990001405809113058130A9F46CE771E081E47E
:1049A00090E00E943B13FC0180819181A281B38140
:1049B0008093BA019093BB01A093BC01B093BD0159
:1049C00010921305809112058130A9F468E771E017
:1049D00086E490E00E943B13FC0180819181A281DA
:1049E000B3818093BA019093BB01A093BC01B093B3
:1049F000BD0110921205809111058130A9F464E780
:104A000071E08BE490E00E943B13FC018081918176
:104A1000A281B3818093BA019093BB01A093BC01A2
:104A2000B093BD0110921105809110058130A9F459
:104A300060E771E080E590E00E943B13FC0180811B
:104A40009181A281B3818093BA019093BB01A0931D
:104A5000BC01B093BD011092100580916405815096
:104A6000873260F480911905813041F460E080E084
:104A70000E94A70986E693E00E945C0A8091640583
:104A8000883260F080911905813041F460E080E067
:104A90000E94A7098BE693E00E945C0A80911905A9
:104AA000811102C01092640580911C0590911D0532
:104AB000019709F098C080910B0590910C05A09189
:104AC0000D05B0910E0585369105A105B105C0F023
:104AD0002AE030E040E050E02093840130938501EB
:104AE00040938601509387018EE690E0A0E0B0E00D
:104AF00080930B0590930C05A0930D05B0930E05C4
:104B000080910B0590910C05A0910D05B0910E05BB
:104B10004F97A109B10986349105A105B105C0F4EB
:104B200022E330E040E050E020938401309385019F
:104B3000409386015093870181E490E0A0E0B0E0CB
:104B400080930B0590930C05A0930D05B0930E0573
:104B500080910B0590910C05A0910D05B0910E056B
:104B60000697A109B1094997A105B105C0F424E64A
:104B700030E040E050E02093840130938501409381
:104B800086015093870181E190E0A0E0B0E080933E
:104B90000B0590930C05A0930D05B0930E05809125
:104BA0000B0590910C05A0910D05B0910E0506978F
:104BB000A105B105C0F428EE33E040E050E02093B9
:104BC00084013093850140938601509387018FE0E3
:104BD00090E0A0E0B0E080930B0590930C05A093CB
:104BE0000D05B0930E058091670590916805892B9E
:104BF00011F40E94EA0A8EE00E943B068EE00E94B9
:104C00003B067C0190931B0580931A056AE070E0D7
:104C100080E090E00E9472068EE00E943B068EE0EB
:104C20000E943B06092E000CAA0BBB0BA7010F2C00
:104C3000000C660B770B4C015D01E3E08E1A9108C6
:104C4000A108B108481559056A057B0564F003966B
:104C5000A11DB11D84179507A607B70724F0F09290
:104C60002F05E0922E05E0902E05F0902F05F5E837
:104C7000EF16F3E0FF060CF462C310921905809161
:104C80001805811106C060E081E10E949F05109225
:104C900066058091880190918901009709F0F8C418
:104CA00021E030E030931D0520931C0524EF31E016
:104CB00040E050E08530910509F011C52093840152
:104CC00030938501409386015093870110921D0512
:104CD00010921C05809167059091680518161906B9
:104CE00014F40E941417809166058130B9F5809103
:104CF000670590916805892B89F5E0901E05F09075
:104D00001F059FEFE91AF90AF0921F05E0921E05B0
:104D100084E10E943B06BC01990F880B990B0E940D
:104D200085302B013C0185E10E943B06BC01990FB7
:104D3000880B990B0E9485304B015C01AC019B01F3
:104D4000C301B2010E94173387FD05C561E080E011
:104D50000E94A70980E793E00E945C0A81E090919D
:104D60006505913009F080E091E020916605211100
:104D700090E0892309F4BFC0809167059091680590
:104D8000892B09F0B8C08091B2019091B301A09134
:104D9000B401B091B501803AE6E89E07E1E0AE07C4
:104DA000B1050CF069C58091BA019091BB01A09149
:104DB000BC01B091BD01805A9648A140B109B0959F
:104DC000A095909581959F4FAF4FBF4F8093300531
:104DD00090933105A0933205B093330580912E0551
:104DE00090912F0587599109C197D0F480912C0596
:104DF00090912D05843691059CF4019690932D0594
:104E000080932C05C29761F4109230051092310501
:104E1000109232051092330510922D0510922C0538
:104E20000E941E0B8091BA019091BB01A091BC0120
:104E3000B091BD014091300550913105609132052E
:104E400070913305840F951FA61FB71F8093B20181
:104E50009093B301A093B401B093B501809128055C
:104E600090912905A0912A05B0912B054817590763
:104E70006A077B07B1F060E375E08FE090E00E9485
:104E8000BA168091300590913105A0913205B0910C
:104E900033058093280590932905A0932A05B093A4
:104EA0002B0561E084E00E94A7096091B201709136
:104EB000B3018091B4019091B50160932405709382
:104EC0002505809326059093270520E432E44FE0E2
:104ED00050E00E94673320932005309321054093D2
:104EE0002205509323050E945E0A80E20E94D809A1
:104EF00080E20E94D8098091660590916505892B12
:104F000009F0FAC08091670590916805892B09F036
:104F1000F3C069E374E08BE996E00E94B4140E9448
:104F2000A3070E94A4060E94A406C0904005D0904A
:104F30004105E0904205F09043056C197D098E090A
:104F40009F09643671058105910540F480913E0505
:104F500090913F0590933D0580933C050E94A406E7
:104F60006C197D098E099F096436710581059105CB
:104F700098F00E94A4066C197D098E099F09683C6F
:104F800071058105910540F480913E0590913F05A2
:104F900090933B0580933A050E94A4066C197D0905
:104FA0008E099F09683C71058105910598F00E9462
:104FB000A4066C197D098E099F096C327140810528
:104FC000910540F480913E0590913F0590933905FD
:104FD000809338050E94A4066C197D098E099F09EB
:104FE0006C3271408105910598F00E94A4066C19FD
:104FF0007D098E099F09603971408105910540F452
:1050000080913E0590913F0590933705809336053A
:105010000E94A4066C197D098E099F0960397140B0
:105020008105910598F00E94A4066C197D098E09EE
:105030009F09653F71408105910540F480913E05CF
:1050400090913F0590933505809334050E94A40606
:105050006C197D098E099F09653F71408105910595
:1050600008F448C080913C0590913D0520913A0597
:1050700030913B05820F931F2091380530913905FF
:10508000820F931F2091360530913705820F931FB1
:105090002091340530913505820F931F65E070E053
:1050A0000E9431337B0170933F0560933E0560EBB6
:1050B00071E083EA90E00E942713FC0180819181D6
:1050C000E816F9060CF4EFC381E993E00E94861418
:1050D00061E084E00E94A7098BE996E00E946404E5
:1050E0000E94A40660934005709341058093420599
:1050F000909343050E941E0B6EE475E084E290E0FD
:105100000E943B13FC0180819181A281B381809335
:105110004A0590934B05A0934C05B0934D0566E46A
:1051200075E085E190E00E943B13FC018081918154
:10513000A281B3818093B6019093B701A093B80187
:10514000B093B90110916605113081F48091BA01D4
:105150009091BB01A091BC01B091BD018093B201BF
:105160009093B301A093B401B093B5018091BA01BB
:105170009091BB01A091BC01B091BD0180389649CE
:10518000A849B10508F461C5809145058111C0C4E5
:1051900066E573E083EB96E00E94B4146DE573E07E
:1051A00087EA96E00E94B41480916505813009F089
:1051B00086C58091B6019091B701A091B801B091D8
:1051C000B9014091B2015091B3016091B401709165
:1051D000B501841B950BA60BB70B80935F059093CD
:1051E0006005A0936105B09362058091440581300C
:1051F00009F0E0C4113009F0DDC480915F059091A1
:105200006005A0916105B091620540914A055091F9
:105210004B0560914C0570914D05841B950BA60BB9
:10522000B70BC0C48EE00E943B06853F91400CF452
:10523000B8C98EE00E943B068A3892400CF48EC8B2
:10524000B0C9D701C6018158934CA94CB1408038F0
:10525000934CA94CB14070F4F694E794D794C7945A
:10526000C092F606D092F706E092F806F092F906A0
:105270006064E2CAD701C60181509748A349B34090
:1052800081159A45A246B24008F0D6CA82E0F6944B
:10529000E794D794C7948A95D1F7C092F606D09236
:1052A000F706E092F806F092F9066068C5CA9130F8
:1052B00009F0D3CB883251F480911405813031F458
:1052C0008CE390E00E94E81410921405809164052C
:1052D000883251F480911305813031F481E490E0FB
:1052E0000E94E8141092130580916405883251F4ED
:1052F00080911205813031F486E490E00E94E81438
:105300001092120580916405883251F48091110544
:10531000813031F48BE490E00E94E8141092110582
:1053200080916405883209F098CB80911005813016
:1053300009F0A4CB80E590E00E94E8148CCB28E42F
:10534000E216F1046CF480911905811109C061E045
:1053500081E10E949F0581E0809366058093190595
:10536000C701895491098D34910538F5809119054B
:10537000811123C08091180581110BC061E081E18A
:105380000E949F0581E080931805809366058093B5
:1053900019058091190581117CCC109118051130E7
:1053A00009F077CC60E081E10E949F05109218051A
:1053B00010926605109319056CCCC70187599109A5
:1053C0008034910508F58091190581111DC08091E7
:1053D0006505811109C081E08093650580931905F9
:1053E00010922D0510922C058091190581110CC089
:1053F00080916505813041F410926505809319050F
:1054000010922D0510922C05C701885D9109C69751
:10541000D8F480911905811117C0809116059091DB
:10542000170501968A3091052CF490931705809307
:10543000160504C0109217051092160581E080939E
:1054400019050E94611325CCC7018F509140C19767
:1054500070F48091190581110AC080911605909110
:105460001705019797FFE1CF89E090E0DECFC701F4
:10547000815491408C97C0F580911905811134C0F9
:1054800080914405811111C061E080E10E949F0577
:1054900011E01093150561E673E08DEA96E00E9435
:1054A000B4141093440510931905809119058111C6
:1054B00014C010914405113081F460E080E10E9435
:1054C0009F051092150568E573E08DEA96E00E944D
:1054D000B414109244051093190565E175E088E055
:1054E00090E00E943B1AD5CBC7018E56914082971F
:1054F000D8F480911905811117C08091450581115B
:1055000005C081E0809345058093190580911905B8
:105510008111BFCB80914505813009F0BACB109243
:10552000450580931905B5CBC701815991408297F4
:10553000F8F48091190581111BC080918801909128
:1055400089010196893091052CF49093890180930B
:10555000880104C0109289011092880181E0809333
:10556000190568E871E087E390E00E94ED1691CBA1
:10557000C701845B91404C9770F4809119058111AB
:105580000AC08091880190918901019797FFDDCF32
:1055900088E090E0DACF9701215D31402337310573
:1055A00008F051C080916405803508F04CC08F5FD1
:1055B0008093640581E0809319052931310558F401
:1055C0008093140510921305109212051092110584
:1055D000109210055ECB97012B5E314029313105C9
:1055E00028F41092140580931305EECF97012550EF
:1055F00032402631310538F410921405109213050B
:1056000080931205E3CF97012C51324024313105AC
:1056100048F410921405109213051092120580930D
:105620001105D6CF9701215332402331310558F46B
:105630001092140510921305109212051092110584
:105640008093100526CB35E4E31A32E0F30A45E4F3
:10565000E416F10408F01DCB80911905811119CBD6
:1056600080916705909168050196909368058093F5
:10567000670521E020930F05099724F01092680533
:105680001092670581E0809319050E94141701CBE1
:105690008130910589F421E030E040E050E0209332
:1056A00084013093850140938601509387011092C5
:1056B0001D0510921C05FACA82309105C1F42AE03A
:1056C00030E040E050E02093840130938501409326
:1056D00086015093870110921D0510921C0586309B
:1056E0009105C1F488EE93E0A0E0B0E023C08330E0
:1056F0009105C1F422E330E040E050E020938401C2
:1057000030938501409386015093870110921D05C7
:1057100010921C0587309105B1F420E137E240E09A
:1057200050E0CCCA8430910509F0C0CA84E690E00C
:10573000A0E0B0E08093840190938501A09386015E
:10574000B0938701C3CA089709F0C4CA80EA96E8F3
:10575000A1E0B0E0EFCFA4E1EA16F1040CF4FECA38
:1057600010921F0510921E05A5019401C301B201FC
:105770000E940A326B017C01A3019201C501B401B0
:105780000E9409329B01AC01C701B6010E9476322A
:105790006B017C0120E030E0A9010E94173318164C
:1057A00024F0F7FAF094F7F8F09420E030E040EAC3
:1057B00050E4C501B4010E94E43020E030EC4FE732
:1057C00054E40E9476322CE238E540EB5CE30E9420
:1057D00076329B01AC010E94E43020E030E048E4E6
:1057E00052E40E9476324B015C0120E030E040E060
:1057F00050E4C701B6010E940A322B013C01A70107
:10580000960160E070E080E89FE30E9476329B01A1
:10581000AC01C301B2010E940A329B01AC0160E0FD
:1058200070E080E890E40E947632A50194010E9425
:10583000E4304B015C0161E080E00E94A70983E84D
:1058400093E00E945C0A42E0C701B6010E94B00BDF
:1058500061E088E00E94A70988E893E00E945C0A62
:1058600061E08BE00E94A70940E0C501B4010E94FD
:10587000B00B8CE893E070CA8138944AAF4BB740C4
:105880000CF4ACCA4091BA015091BB016091BC01CB
:105890007091BD0180E894EAAFEBB7E0841B950BF3
:1058A000A60BB70B93CA60EB71E083EA90E00E940D
:1058B0002713DC018D919C918E159F051CF48EE9B8
:1058C00093E004CC6EEA71E080EA90E00E94271336
:1058D000FC01808191818E159F051CF48BEA93E079
:1058E000F5CB6CEA71E08DE990E00E942713DC01B2
:1058F0008D919C918E159F051CF488EB93E0E6CB6F
:105900006AEA71E08AE990E00E942713FC01808135
:1059100091818E159F051CF485EC93E0D7CB68EA46
:1059200071E087E990E00E942713DC018D919C9142
:105930008E159F051CF482ED93E0C8CB66EA71E0FA
:1059400084E990E00E942713FC01808191818E15EB
:105950009F051CF48FED93E0B9CB64EA71E081E917
:1059600090E00E942713DC018D919C918E159F057C
:105970001CF48CEE93E0AACB62EA71E08EE890E032
:105980000E942713FC01808191818E159F051CF4D4
:1059900089EF93E09BCB60EA71E08BE890E00E9496
:1059A0002713DC018D919C918E159F051CF486E0D8
:1059B00094E08CCB6EE971E088E890E00E942713B8
:1059C000FC01808191818E159F051CF483E194E098
:1059D0007DCB6CE971E085E890E00E942713DC0143
:1059E0008D919C918E159F051CF480E294E06ECB06
:1059F0006AE971E082E890E00E942713FC0180814F
:105A000091818E159F051CF48DE294E05FCB68E9CF
:105A100071E08FE790E00E942713DC018D919C914B
:105A20008E159F051CF48AE394E050CB66E971E083
:105A30008CE790E00E942713FC01808191818E15F4
:105A40009F051CF487E494E041CB64E971E089E7A9
:105A500090E00E942713DC018D919C918E159F058B
:105A60001CF484E594E032CB62E971E086E790E0D3
:105A70000E942713FC01808191818E159F051CF4E3
:105A800081E694E023CB60E971E083E790E00E9437
:105A90002713DC018D919C918E159F051CF48EE6D9
:105AA00094E014CB6EE871E080E790E00E94271349
:105AB000FC01808191818E159F051CF48BE794E099
:105AC00005CB6CE871E08DE690E00E942713DC01C5
:105AD0008D919C918E159F051CF488E894E0F6CA80
:105AE0006AE871E08AE690E00E942713FC01808159
:105AF00091818E159F051CF485E994E0E7CA6AE858
:105B000071E087E690E00E94271382EA94E0DECA03
:105B1000813009F09AC06FEA74E083EB96E00E944E
:105B2000B41461EB74E087EA96E00E94B4148091AB
:105B30006505813009F0A4C08091B6019091B7014C
:105B4000A091B801B091B9014091B2015091B30157
:105B50006091B4017091B501841B950BA60BB70B36
:105B600080935F0590936005A0936105B0936205F3
:105B7000809144058130F1F41130E1F480915F05AA
:105B800090916005A0916105B091620540914A0530
:105B900050914B0560914C0570914D05840F951FF8
:105BA000A61FB71F80935F0590936005A0936105C2
:105BB000B093620580916305811105C060E081E0CA
:105BC00090E00E94380880916305813009F038C167
:105BD00061E081E090E00E94380840915F055091BB
:105BE0006005609161057091620580915B059091FF
:105BF0005C05A0915D05B0915E05481759076A07DD
:105C00007B0709F0FBC02091AB063091AC06809178
:105C1000A5069091A6062817390709F0EFC08091D4
:105C2000A7069091A8066091A1067091A206009720
:105C300009F4D7C06115710509F054C0232B09F48C
:105C4000FFC0FC01808190E0D7C08091BA019091A3
:105C5000BB01A091BC01B091BD0180389649A84913
:105C6000B10508F0A7CF8091450581111CC06FEAEE
:105C700074E083EB96E00E94B4146DE573E053CFBB
:105C8000811176CF4091BA015091BB016091BC0166
:105C90007091BD018091B6019091B701A091B801BA
:105CA000B091B90159CF813009F084CF66E573E036
:105CB00083EB96E00E94B41461EB74E071CA811129
:105CC00094CA4091BA015091BB016091BC0170919E
:105CD000BD018091B6019091B701A091B801B0913A
:105CE000B90177CA0E94113787C081EA96E00E9405
:105CF0001013A6C00E94C2358AA19BA1909396065C
:105D0000809395068CA19DA1909398068093970609
:105D10008EA19FA190939A06809399061BA21AA226
:105D20001DA21CA22BC185E996E00E94101366C13A
:105D300064E670E080E090E00E94720660915F058A
:105D400070916005809161059091620524E630E0D4
:105D500040E050E00E94ED3310E000E00E94F40EBD
:105D600080915F0590916005A0916105B0916205F9
:105D700080935B0590935C05A0935D05B0935E05F1
:105D80008091BA019091BB01A091BC01B091BD017D
:105D90008093520590935305A0935405B0935505F5
:105DA0008091670590916805892B59F4809164056D
:105DB000811107C060E00E94A7098DEA96E00E9469
:105DC000640480E090E0892B11F40C94A7240E94D5
:105DD000AA04882311F40C94A7240E9400000C94B8
:105DE000A7246115710561F1232B51F1DB018C9121
:105DF00090E0919581959109892B11F16091BA01FB
:105E00007091BB018091BC019091BD0124E630E00E
:105E100040E050E00E94ED3301E010E00E94F40EFB
:105E20006091A7067091A8066115710509F45DCF10
:105E30004091AB065091AC0681EA96E00E94931423
:105E400080915A05811105C060E082E090E00E94D7
:105E5000380880915A058130A1F561E082E090E038
:105E60000E9438086091B6017091B7018091B80125
:105E70009091B901C0905605D0905705E090580513
:105E8000F09059056C157D058E059F05D1F024E62F
:105E900030E040E050E00E94DE3302E010E00E947B
:105EA000F40E8091B6019091B701A091B801B09124
:105EB000B9018093560590935705A0935805B09368
:105EC000590540915F0550916005609161057091A1
:105ED000620580915B0590915C05A0915D05B09194
:105EE0005E05481759076A077B0709F459CF809167
:105EF000670590916805892B09F052CF8FE190E0FA
:105F00000E94E8140E9411156091BA017091BB01C2
:105F10008091BC019091BD011BA21AA21DA21CA2DE
:105F20001FA21EA22AE0AE014F5F5F4F0E943230D7
:105F3000BE016F5F7F4FCE0182960E94B4148091A4
:105F4000950690919606009709F4D6CE6AA17BA19A
:105F50006115710509F4CECE4091970650919806CF
:105F60002EA13FA14217530708F4C4CE0E941A374E
:105F70008EA19FA190939A06809399061FA21EA2BC
:105F8000CE0182960E9422138091990690919A06E2
:105F90000B9708F0CDCE1BA21AA21DA21CA21FA215
:105FA0001EA24AE0BE016F5F7F4F90E080E00E943A
:105FB0002730BE016F5F7F4FCE0182960E94B414DE
:105FC0004091990650919A066091950670919606B7
:105FD000CE0182960E945A14811104C0CE0182968D
:105FE0000E9410136AA17BA16115710509F49BCE73
:105FF0004EA15FA185E996E00E949314CE0182969E
:106000000E942213C1CF83E896E00E94221389E800
:1060100096E00E9422138FE896E00E94221385E901
:1060200096E00E9422138BE996E00E94221381EAF7
:1060300096E00E94221387EA96E00E9422138DEADE
:1060400096E00E94221383EB96E00C942213BB2768
:106050004A3031F4992322F4BDE2909581959F4F07
:106060000C945530BB27FA01A62F621771058105E4
:106070009105330B30FB66F0AA27660F771F881F48
:10608000991FAA1FA21710F0A21B63953850A9F7F9
:10609000A05DAA3308F0A95DA19336F7B111B193C1
:1060A0001082CA010C946E30BB27FB015527AA272A
:1060B000880F991FAA1FA41710F0A41B8395505195
:1060C000B9F7A05DAA3308F0A95DA193009779F70D
:1060D000B111B1931192CB010C946E30DC01FC0133
:1060E000672F71917723E1F7329704C07C916D930C
:1060F00070836291AE17BF07C8F308950E94C03045
:1061000008F481E00895E89409C097FB3EF4909567
:106110008095709561957F4F8F4F9F4F9923A9F080
:10612000F92F96E9BB279395F6958795779567950F
:10613000B795F111F8CFFAF4BB0F11F460FF1BC053
:106140006F5F7F4F8F4F9F4F16C0882311F096E9E6
:1061500011C0772321F09EE8872F762F05C0662394
:1061600071F096E8862F70E060E02AF09A95660F4D
:10617000771F881FDAF7880F9695879597F9089506
:10618000990F0008550FAA0BE0E8FEEF1616170648
:10619000E807F907C0F012161306E407F50798F0B0
:1061A000621B730B840B950B39F40A2661F0232BC9
:1061B000242B252B21F408950A2609F4A140A69545
:1061C0008FEF811D811D08950E94F7300C94683176
:1061D0000E945A3138F00E94613120F0952311F06D
:1061E0000C9451310C94573111240C949C310E9421
:1061F000793170F3959FC1F3950F50E0551F629F61
:10620000F001729FBB27F00DB11D639FAA27F00D0F
:10621000B11DAA1F649F6627B00DA11D661F829F36
:106220002227B00DA11D621F739FB00DA11D621F1B
:10623000839FA00D611D221F749F3327A00D611D38
:10624000231F849F600D211D822F762F6A2F11241A
:106250009F5750409AF0F1F088234AF0EE0FFF1F4D
:10626000BB1F661F771F881F91505040A9F79E3FA4
:10627000510580F00C9451310C949C315F3FE4F354
:10628000983ED4F3869577956795B795F795E795FA
:106290009F5FC1F7FE2B880F911D9695879597F903
:1062A000089597F99F6780E870E060E008959FEF98
:1062B00080EC089500240A9416161706180609069D
:1062C000089500240A94121613061406050608956C
:1062D000092E0394000C11F4882352F0BB0F40F4F4
:1062E000BF2B11F460FF04C06F5F7F4F8F4F9F4F34
:1062F000089557FD9058440F551F59F05F3F71F0B6
:106300004795880F97FB991F61F09F3F79F087951C
:106310000895121613061406551FF2CF4695F1DFA5
:1063200008C0161617061806991FF1CF8695710535
:10633000610508940895E894BB2766277727CB0169
:1063400097F90895F999FECF92BD81BDF89A9927E2
:1063500080B50895262FF999FECF1FBA92BD81BD51
:1063600020BD0FB6F894FA9AF99A0FBE01960895D7
:106370000E94FA31A59F900DB49F900DA49F800DAF
:10638000911D112408952F923F924F925F926F9228
:106390007F928F929F92AF92BF92CF92DF92EF92B5
:1063A000FF920F931F93CF93DF93CDB7DEB7CA1B36
:1063B000DB0B0FB6F894DEBF0FBECDBF09942A8861
:1063C000398848885F846E847D848C849B84AA8409
:1063D000B984C884DF80EE80FD800C811B81AA8196
:1063E000B981CE0FD11D0FB6F894DEBF0FBECDBF61
:1063F000ED010895A29FB001B39FC001A39F700D4E
:10640000811D1124911DB29F700D811D1124911DBC
:1064100008955058BB27AA270E9421320C94683156
:106420000E945A3138F00E94613120F039F49F3FC8
:1064300019F426F40C9457310EF4E095E7FB0C9414
:106440005131E92F0E94793158F3BA176207730767
:106450008407950720F079F4A6F50C949B310EF48F
:10646000E0950B2EBA2FA02D0B01B90190010C0164
:10647000CA01A0011124FF27591B99F0593F50F47C
:10648000503E68F11A16F040A22F232F342F4427D4
:10649000585FF3CF469537952795A795F0405395CC
:1064A000C9F77EF41F16BA0B620B730B840BBAF09C
:1064B0009150A1F0FF0FBB1F661F771F881FC2F707
:1064C0000EC0BA0F621F731F841F48F4879577951B
:1064D0006795B795F7959E3F08F0B0CF9395880FD5
:1064E00008F09927EE0F9795879508950E948A32B4
:1064F0000C9468310E94613158F00E945A3140F08A
:1065000029F45F3F29F00C94513151110C949C31C6
:106510000C9457310E94793168F39923B1F35523D4
:1065200091F3951B550BBB27AA27621773078407A6
:1065300038F09F5F5F4F220F331F441FAA1FA9F33C
:1065400035D00E2E3AF0E0E832D091505040E6952A
:10655000001CCAF72BD0FE2F29D0660F771F881F8B
:10656000BB1F261737074807AB07B0E809F0BB0B7E
:10657000802DBF01FF2793585F4F3AF09E3F510592
:1065800078F00C9451310C949C315F3FE4F3983EC9
:10659000D4F3869577956795B795F7959F5FC9F77B
:1065A000880F911D9695879597F90895E1E0660FFC
:1065B000771F881FBB1F621773078407BA0720F075
:1065C000621B730B840BBA0BEE1F88F7E0950895DE
:1065D0000E94813188F09F5798F0B92F9927B751C1
:1065E000B0F0E1F0660F771F881F991F1AF0BA9577
:1065F000C9F714C0B13091F00E949B31B1E0089509
:106600000C949B31672F782F8827B85F39F0B93FFA
:10661000CCF3869577956795B395D9F73EF4909529
:106620008095709561957F4F8F4F9F4F08950E9481
:10663000C03008F48FEF08950E94C030880B990B8A
:106640000895DB018F939F930E94B831BF91AF9162
:10665000A29F800D911DA39F900DB29F900D1124BC
:10666000089597FB072E16F4009407D077FD09D004
:106670000E940C3507FC05D03EF4909581959F4F04
:106680000895709561957F4F0895A1E21A2EAA1B77
:10669000BB1BFD010DC0AA1FBB1FEE1FFF1FA217D2
:1066A000B307E407F50720F0A21BB30BE40BF50BCF
:1066B000661F771F881F991F1A9469F76095709558
:1066C000809590959B01AC01BD01CF010895052EE9
:1066D00097FB1EF400940E947E3357FD07D00E9462
:1066E000453307FC03D04EF40C947E33509540950F
:1066F000309521953F4F4F4F5F4F0895909580956E
:10670000709561957F4F8F4F9F4F0895DF93CF9383
:106710001F930F939A9DF02D219FF00D8B9DF00DEF
:106720008A9DE02DF10D039FF00D029FE00DF11DFC
:106730004E9DE00DF11D5E9DF00D4F9DF00D7F9380
:106740006F93BF92AF925F934F93D5010E94FA313E
:106750008B01AC01D7010E94FA31EB01E80FF91F60
:10676000D6010E94D5332F913F91D6010E94FA3174
:10677000C60FD71FE81FF91FAF91BF910E94D533F5
:106780002F913F910E94FA31C60FD71FE81FF91FC2
:10679000D6010E94FA31E60FF71F9801BE01CF0122
:1067A0000F911F91CF91DF9108950E94FA31460F0A
:1067B000571FC81FD91F08F43196089597FB57FF3C
:1067C0000C94EE339F938F930E94EE336E1B7F0BDE
:1067D000AF91BF918A0B9B0B0895E894DF93CF9301
:1067E000FC01DB010E94FA317F936F93E9019A016A
:1067F000AC01BF93AF933F932F93DF010E94FA3117
:1068000026F46C1B7D0B820B930B9E01EB01FC01AC
:106810000E94D533AF91BF912F913F910E94D53304
:10682000BE01CF01F9012F913F91CF91DF910895E2
:10683000689401C0E894F92FF12B12F00C944C34B9
:10684000A0E0B0E0E6E2F4E30C94C931092E05942F
:1068500022F40E94A834112392F4F0E80F26FFEFEF
:10686000E094F09400951095B094C094D094A194C5
:10687000BF0ACF0ADF0AEF0AFF0A0F0B1F0B0E94A5
:10688000573407FC0E94A834CDB7DEB7ECE00C9477
:10689000E531689401C0E8948F929F92CF93DF9383
:1068A0000E945734DF91CF919F908F900895882454
:1068B0009924F401E401B0E49F93AA279A158B046C
:1068C0009C04ED05FE05CF05D007A10798F4AD2F78
:1068D000DC2FCF2FFE2FE92D982C892E982F872F74
:1068E000762F652F542F432F322F2227B85031F7A0
:1068F000BF9127C01B2EBF91BB27220F331F441F00
:10690000551F661F771F881F991F881C991CEE1F33
:10691000FF1FCC1FDD1FAA1FBB1F8A149B04EC05A1
:10692000FD05CE05DF05A007B10748F08A189B08D2
:10693000EC09FD09CE09DF09A00BB10B21601A9407
:10694000E1F62EF49401AF01BE01CD01000C0895D3
:1069500060957095809590953095409550952195CE
:106960003F4F4F4F5F4F6F4F7F4F8F4F9F4F089558
:10697000002E083090F0982F872F762F652F542FF8
:10698000432F322F22270850F4CF220F331F441FEA
:10699000551F661F771F881F991F0A95B2F7002D94
:1069A000089597FD1094002E083098F00850232F7A
:1069B000342F452F562F672F782F892F912DF4CF05
:1069C000159497958795779567955795479537953A
:1069D00027950A95AAF71124002D08952A0D3B1D2D
:1069E0004C1D5D1D6E1D7F1D801F911F08952A1572
:1069F0003B054C055D056E057F05800791070895F1
:106A00000024A7FD00942A173005400550056005B5
:106A10007005800590050895AA1BBB1B51E107C0B6
:106A2000AA1FBB1FA617B70710F0A61BB70B881F1E
:106A3000991F5A95A9F780959095BC01CD010895AD
:106A4000EE0FFF1F0590F491E02D09940F931F9313
:106A5000CF93DF938230910510F482E090E0E091D3
:106A60001407F091150730E020E0B0E0A0E0309787
:106A700099F42115310509F44AC0281B390B24303B
:106A80003105D8F58A819B816115710589F1FB017A
:106A900093838283FE0111C0408151810281138161
:106AA00048175907E0F04817590799F4109761F013
:106AB00012960C93129713961C933296CF01DF9186
:106AC000CF911F910F91089500931407109315070C
:106AD000F4CF2115310551F04217530738F0A901C1
:106AE000DB019A01BD01DF01F801C1CFEF01F9CF50
:106AF0009093150780931407CDCFFE01E20FF31F8B
:106B0000819391932250310939832883D7CF2091E3
:106B1000120730911307232B41F42091C0013091CB
:106B2000C10130931307209312072091BE013091C9
:106B3000BF012115310541F42DB73EB74091C20187
:106B40005091C301241B350BE0911207F0911307FC
:106B5000E217F307A0F42E1B3F0B2817390778F034
:106B6000AC014E5F5F4F2417350748F04E0F5F1F93
:106B70005093130740931207819391939FCFF0E0B6
:106B8000E0E09CCFCF93DF930097E9F0FC013297D0
:106B900013821282A0911407B0911507ED0130E025
:106BA00020E01097A1F420813181820F931F209162
:106BB0001207309113072817390709F061C0F093C5
:106BC0001307E0931207DF91CF910895EA01CE17E2
:106BD000DF07E8F54A815B819E0141155105B1F758
:106BE000E901FB83EA8349915991C40FD51FEC1742
:106BF000FD0761F4808191810296840F951FE90160
:106C000099838883828193819B838A83F0E0E0E08B
:106C100012968D919C9113970097B9F52D913C9107
:106C20001197CD010296820F931F20911207309188
:106C300013072817390739F6309751F510921507C1
:106C400010921407B0931307A0931207BCCFD383FD
:106C5000C28340815181840F951FC817D90761F401
:106C60004E5F5F4F88819981480F591F5183408340
:106C70008A819B81938382832115310509F0B0CFEE
:106C8000F0931507E09314079ECFFD01DC01C0CF00
:106C900013821282D7CFB0E0A0E0E1E5F6E30C94D6
:106CA000C5318C01009751F4CB010E9426358C012F
:106CB000C801CDB7DEB7E0E10C94E131FC01E60F8D
:106CC000F71F9C0122503109E217F30708F49DC019
:106CD000D901CD91DC911197C617D70798F0C5302F
:106CE000D10530F3CE0104978617970708F3C61B2A
:106CF000D70B2297C193D1936D937C93CF010E94C0
:106D0000C235D6CF5B01AC1ABD0A4C018C0E9D1E5C
:106D1000A0911407B0911507512C412CF12CE12CB6
:106D2000109731F5809112079091130788159905F6
:106D300009F05CC04616570608F058C08091BE01A5
:106D40009091BF01009741F48DB79EB74091C20169
:106D50005091C301841B950BE817F90708F055C043
:106D6000F0931307E0931207F90171836083A0CFBA
:106D70008D919C91119712966C90129713967C901E
:106D80001397A815B90559F56C0142E0C40ED11C42
:106D9000CA14DB0420F1AC014A195B09DA0112962E
:106DA000159780F06282738251834083D9016D937D
:106DB0007C93E114F10471F0D7011396FC93EE93E8
:106DC000129776CF22968C0F9D1FF90191838083B5
:106DD000F301EFCFF0931507E093140769CF48163E
:106DE000590608F42C017D01D3019ACFCB010E94F2
:106DF00026357C01009749F0AE01B8010E940837A2
:106E0000C8010E94C235870153CF10E000E050CF87
:106E1000FB01DC0102C001900D9241505040D8F7B7
:106E20000895FB01DC018D91019080190110D9F3C7
:106E3000990B0895FB01DC0101900D920020E1F710
:106E4000089510E0C2E6D0E004C0FE010E942035A3
:0C6E50002196C336D107C9F7F894FFCF94
:106E5C0070E9D700C0320A0320E0B201903B7E01FA
:106E6C00D03F4401407D140170E9D700406B9A007B
:106E7C0010936B00D0B13700903A1C0079003C00A5
:106E8C0040787D01503403001F1115111D1D111F79
:106E9C001F1115111515111F1F111D1D1D1D1D1F56
:106EAC001F1117111515111F1F1117111D1D111F62
:106EBC001F1515111D1D1D1F1F111D111D1D111F2E
:106ECC0070E9D70070E09A00B0196D00D0B13700AE
:106EDC00903A1C00F401000005009301BE01EA0188
:106EEC00FE01120226023A026C02BA02E4020C0300
:106EFC0048035C03720388039D03A103A403A80346
:106F0C00AC0340420F0080F0FA0270E9D700000099
:106F1C0016078000000204000300011003020000A9
:106F2C00030201000600040006050020060504000B
:106F3C0000000000E00437046D042D059E047C0461
:106F4C0090040000000031070407A007E106EA00E6
:106F5C00F106E20600000000B6093704A00736046B
:106F6C0031487A20003130487A003530487A003187
:106F7C00303048003530304800316B487A003130C1
:106F8C006B48003130306B004175746F006E616E70
:106F9C0000696E66006F766600436F72722E504CFD
:106FAC004C205369353335312020002020436F723B
:106FBC00726563742E2042464F2020002020202032
:106FCC0020434C4B202D203220202020004F666681
:106FDC00004F6E20002056464F2D3E20434C4B2D2B
:106FEC0031200020436F72722E2053686966742022
:106FFC0043572000487A202020202000436F7272D3
:10700C00465245512E2051554152545A0020487A2F
:10701C0000436F72722E20535F4C4556454C202D09
:10702C003F00202050494E204130203D2000302090
:10703C0042616C6C203D204F46462056464F200046
:10704C00332042616C6C3D20302E38206D6B562005
:10705C0000362042616C6C3D2036206D6B56202032
:10706C002000392042616C6C3D203530206D6B5610
:10707C00202000392B323064423D20353030206DD9
:10708C006B562000392B343064423D203530303083
:10709C00206D6B5600392B363064423D2035303034
:1070AC0030306D6B5600550053534220004C534208
:1070BC000043572020004C4F4144005245432000D0
:1070CC00535752202020202020503D305720202084
:1070DC002020005357523D0020503D0057202020C7
:1070EC0000FFFFFFFFFFFFFFFF072B363000FFFF06
:1070FC00FFFFFFFFFFFF072B353500FFFFFFFFFFF3
:10710C00FFFFFF072B353000FFFFFFFFFFFFFFFFE7
:10711C00072B343500FFFFFFFFFFFFFFFF072B346A
:10712C003000FFFFFFFFFFFFFFFF072B333500FF92
:10713C00FFFFFFFFFFFFFF072B333000FFFFFFFFB9
:10714C00FFFFFFFF072B323500FFFFFFFFFFFFFFA5
:10715C00FF072B323000FFFFFFFFFFFFFFFF072B66
:10716C00313500FFFFFFFFFFFFFFFF072B31300022
:10717C00FFFFFFFFFFFFFFFF072B352000FFFFFF87
:10718C00FFFFFFFFFF0720202000FFFFFFFFFFFF97
:10719C00FF062020202000FFFFFFFFFFFF0520201F
:1071AC0020202000FFFFFFFFFF04202020202020B4
:1071BC0000FFFFFFFF032020202020202000FFFFE6
:1071CC00FF02202020202020202000FFFF01202073
:1071DC002020202020202000FFFF20202020202005
:1071EC002020202000FF20202020202020202020D4
:1071FC002000202020202020202020202020004C97
:06720C0000555342000092
:00000001FF
